:10530300506C6561736520696E73657274206D6F8F
:1053130064756C6500202755696E202B2D3130563E
:1053230027202830783631292000202020202069AA
:105333006E746F20706F7274203020202020002044
:10534300202027446F757427202830783430292093
:105353002020200020202020696E746F20706F723F
:1053630074203120202020200020002A2A20002021
:105373002A2A00202020416464726573733A202036
:10538300253034580020205265766973696F6E3A70
:10539300202025730057726F6E672043504C4420C2
:1053A3006669726D7761726500536C617665206121
:1053B3006464723A20256264005265713A20253094
:1053C30032626420213D204163743A2025303262E9
:1053D30064004F76657263757272656E74203E3138
:1053E3002E3541206F6E00202020323456206F75F9
:1053F3007470757420212121202020002020205347
:105403006C61766520616464723A2025626400529F
:1054130045534554004F76657263757272656E74B9
:10542300203E302E3541206F6E002020202035563F
:10543300206F757470757420212121002020202095
:10544300536C61766520616464723A20256264005E
:105453002020202055203D2025312E326620560065
:10546300414443303A2025312E33662056004144CF
:1054730043313A2025312E3366205600564152538C
:10548300005343532D323030312D415050002449C5
:10549300643A207363735F323030305F6170702E13
:1054A30063203238373420323030352D31312D31CD
:1054B300352030383A34373A31345A2072697474AB
:1054C3002024000418000001414443303000000050
:1054D300010B4C040000000000000000000000006D
:1054E3000000000418000001414443303100000073
:1054F300010B500400000000000000000000000049
:105503000000000418000001414443303200000051
:10551300010B540400000000000000000000000024
:105523000000000418000001414443303300000030
:10553300010B580400000000000000000000000000
:10554300000000041800000141444330340000000F
:10555300010B5C04000000000000000000000000DC
:1055630000000004180000014144433035000000EE
:10557300010B6004000000000000000000000000B8
:1055830000000004180000014144433036000000CD
:10559300010B640400000000000000000000000094
:1055A30000000004180000014144433037000000AC
:1055B300010B680400000000000000000000000070
:1055C300000000013200000056616C766530000077
:1055D300010B6C00000000003F8000003F800000D2
:1055E300000000013200000056616C766531000056
:1055F300010B6D00000000003F8000003F800000B1
:10560300000000013200000056616C766532000034
:10561300010B6E00000000003F8000003F8000008F
:10562300000000013200000056616C766533000013
:10563300010B6F00000000003F8000003F8000006E
:10564300000000013200000056616C7665340000F2
:10565300010B7000000000003F8000003F8000004D
:10566300000000013200000056616C7665350000D1
:10567300010B7100000000003F8000003F8000002C
:10568300000000013200000056616C7665360000B0
:10569300010B7200000000003F8000003F8000000B
:1056A300000000013200000056616C76653700008F
:1056B300010B7300000000003F8000003F800000EA
:1056C30000000000000000000000000000000000D7
:1056D30000000000000000000000000000000000C7
:0356E300000000C4
:10A81A00017801031CFF54C6C111C10CC112C11336
:08A82A00C10DC10EC10FC110E8
:108F5B0075840F75A4F575A5FF75A6FF75A70FE4AE
:108F6B00F584F5BA75BC9875E880F5D1F58475D1A3
:108F7B0003F58475D48075840175D480FDFF12AC24
:108F8B00837B61E4FDFF12A8CAEF70297BFF7A5344
:108F9B007903124EF67BFF7A537918124EF67BFF4C
:108FAB007A53792D124EF6E4FF12A41FEF7006FFD1
:108FBB0012AA2880F27B407D01E4FF12A8CAEF7051
:108FCB00297BFF7A537903124EF67BFF7A53794252
:108FDB00124EF67BFF7A537957124EF6E4FF12A42A
:108FEB001FEF7006FF12AA2880F212A178157015D8
:108FFB00701570A87076000876000876001570A8BA
:10900B0070E4F61570A870F6FB7D017F611256E6D1
:10901B00157015701570A87076000876000876002C
:10902B001570A870E4F61570A8707601FB7D017FB2
:04903B0040027CA3D0
:0284AF008F44F8
:1084B1007D017F0012A99E7D007F0112A99EE4909B
:1084C1000C16F0900C16E0FFC39403500B12939C12
:1084D100900C16E004F080EB12AD3BE4900C16F02A
:1084E100900C16E0FFC39408500FEF2408FF12AC64
:1084F10027900C16E004F080E7E4FDFF12AC83E462
:10850100900C16F07B007A00799312000E7C007DAE
:10851100021207E9C374079FFFE49EFE900C16E068
:10852100C39FEE6480F874809850117BFF7A537971
:108531006C12AAAA900C16E004F080C87BFF7A5353
:10854100796E12AAAA7B007A00799312AAAA7BFFFC
:108551007A53797212AAAA7D01E4FF12AC837BFFE0
:108561007A537976788DE6F54808E6F549124EF6A4
:108571007D02E4FF12AC83900C16740AF07BFF7A43
:1085810054799112000E900C16E0FDC39FEE6480A9
:10859100F87480985011ED90549193642060089084
:1085A1000C16E004F080D6900C16E02492F9E43425
:1085B100547548FFF549894A754B00754C067B0196
:1085C1007A0C791712A5227B017A0C79177D20127A
:1085D100ABBEE412074E75480175490C754A177B0D
:0885E100FF7A537988024EF67F
:10A41F00E4F58420110FD211F58475D103F5BA75C7
:0DA42F00BC9875E880C374079F5407F5BB07
:0DA43C0075440275451300D545FCD544F666
:10A44900C2AFC2EDD2EC30EDFDD2AFAFBFEFFFAD81
:10A45900BEED900C31CFF0A3EFF0C3E094E8900C7F
:0CA4690031E0940350047F0180027F006A
:01A4750022C4
:106A3D00E4900C2AF012ACBDC8ECC8C9EDC9CAEE81
:106A4D00CACBEFCB900B08E0FCA3E0FDA3E0FEA3C7
:106A5D00E0240AFFE43EFEE43DFDE43CFCD31208D5
:106A6D00FD501A12ACBD900B08E0F8A3E0F9A3E0BD
:106A7D00FAA3E0FBD31208FD5003026CDB12ACBD90
:106A8D00900B08120A08E4900C2BF0900C2BE0FFF1
:106A9D00C394014003026CEA7B017A0C7929129AA6
:106AAD001C900C29E0C4540F640260617A007B6471
:106ABD007D017F01129B4020134B12AD15E4FDFFAC
:106ACD0012AC837BFF7A53799812AAAA7D01E4FF59
:106ADD0012AC83900C2BE0FFD39400400B7BFF7A1C
:106AED005379AC8F48124EF67D02E4FF12AC837BD6
:106AFD00FF7A5379BC754802900C29E0FFC4540FFE
:106B0D00F549124EF6D213900C2A7401F0900C2B0D
:106B1D00E0FF75420175430C75442C754503E4FB8C
:106B2D007D01128374900C2CE020E303026BBD7A7F
:106B3D00007B647D017F01129B4020124E12AD152A
:106B4D00E4FDFF12AC837BFF7A5379D5124EF67DAF
:106B5D0001E4FF12AC837BFF7A5379EA124EF67D86
:106B6D0002E4FF12AC83900C2BE0FFD39400400B9A
:106B7D007BFF7A5379FF8F48124EF67D037F0F12FC
:106B8D00AC837BFF7A547912124EF6D2127F031228
:106B9D00A41FEF6015900C2BE0FF12AB83C2127F88
:106BAD000312A41FEF70F812AD15900C2A7401F0AA
:106BBD0012ACBDE47B64FAF9F8C31208FD40030280
:106BCD006CD2900C2BE0FF75420175430C75442F70
:106BDD007545027B037D02128374900C2FE0C4F87F
:106BED0054F0C868FCA3E0C4540F48FDE41203B68A
:106BFD00E4FBFA79C8784012019EE4FBFA798078BB
:106C0D00451202A7E4FBFA79907840120344600222
:106C1D005003026CBE200C4912AD157A007B647DC9
:106C2D00017F01129B40E4FDFF12AC837BFF7A5480
:106C3D007918124EF67D01E4FF12AC837BFF7A5476
:106C4D00792D124EF67D02E4FF12AC83900C2BE0F1
:106C5D00FFD39400400B7BFF7A54793F8F48124E3F
:106C6D00F67D03E4FF12AC83900C2FE0C4F854F0D2
:106C7D00C868FCA3E0C4540F48FDE41203B6E4FB5E
:106C8D00FA79C8784012019EE4FBFA7980784512B2
:106C9D0002A78F4B8E4A8D498C487BFF7A547953CE
:106CAD00124EF6D20C900B747401F0900C2AF080F9
:106CBD0014300C11900C2BE0FF900B74E06F7005ED
:106CCD00C20C12AD15900C2BE004F0026A98201244
:106CDD0006200C03301306900C2A7401F0900C2A38
:026CED00E0FFC6
:016CEF002282
:10AC27001570A870EFF6A870E6240CF582E4340BD3
:08AC3700F5837401F0057022A1
:05AD49008F397F00229C
:10A9CE008B398A3A893B120708AB3CAA3DA93E1245
:10A9DE00074EAB39AA3AA93B900001120721AB3CB6
:0DA9EE00AA3DA93E9000011207607F0222E1
:109FA20030140312AD15E4FDFF12AC837BFF7A542B
:109FB2007963900B4CE0FCA3E0FDA3E0FEA3E0F587
:109FC2004B8E4A8D498C48124EF67D01E4FF12AC4D
:109FD200837BFF7A547971900B50E0FCA3E0FDA3E0
:109FE200E0FEA3E0F54B8E4A8D498C48124EF67D79
:109FF20003E4FF12AC837BFF7A54797F124EF62082
:10A002001409200806300D037F0122A208920DA236
:0EA0120009920EA20A920FA20B92107F00225A
:10A93700E4FFFEFD7C40900B4CE0F8A3E0F9A3E0B8
:10A94700FAA3E0FB120344600A4008900B6C740101
:10A95700F08005E4900B6CF07E08CFEECF12AC27A9
:04A967000EBE0FF61B
:01A96B0022C9
:08000300C2AF120971D2AF2255
:108D8200900C167408F0900C16E0FFC3940F504B31
:108D9200740C2FF582E4340BF583E06036900C16E8
:108DA200E0240CF582E4340BF583E4F015701570C1
:108DB2001570A870760108760B08766CEF24F8150A
:108DC20070A870F61570A87076017B007D027F4056
:108DD200127CA3900C16E004F080ABE4900C16F029
:108DE200900C16E0FFC39408505915701570157059
:108DF200A870760108760C0876181570A870EFF640
:108E02001570A870E4F6FB7D037F611256E6900CA4
:108E120017EFF0D394004023900C16E075F004A4F1
:108E2200244CF9740B35F0FA7B01900C18E0FCA38A
:108E3200E0FDA3E0FEA3E0FF120003900C16E004A5
:108E4200F0809D12A937E4FF12A41FEF24FF9208BD
:108E52007F0112A41FEF24FF92097F0212A41FEFC9
:108E620024FF920A7F0312A41FEF24FF920B020B2E
:018E7200956A
:10617D00202020202020202020200025622A62645B
:10618D000025622A62750025622A640025622A753F
:10619D000025622A2E622A660025622A6C6400257B
:1061AD00622A6C7500253262753A25730020202015
:1061BD002020202020004E6F207661726961626C74
:1061CD00657320646566696E65640020202020205B
:1061DD0020202020202020202020202020200045AD
:1061ED00534320454E5445522020202D2020202061
:1061FD002B20200045534320454E5445522020204E
:10620D002D20202020202B200045534320454E5487
:10621D0045522020200045534320202020202020BF
:10622D002020002020202020002000506172616D70
:10623D006574657273207772697474656E00746F1E
:10624D0020666C617368206D656D6F72792E00F438
:10625D0070000000F76E000000FA8F000000FD6D69
:10626D000000000000000000036B000000064D0060
:10627D00000009470000000C5400000063000000FE
:10628D0000016D00000002670000000373000000B4
:10629D00046D0000000568000000064100000007C5
:1062AD004B000000088043000009804600001448A0
:1062BD007A0000155061000016626100001757004A
:1062CD000000185600000019B50000001A54000017
:1062DD00001B6C2F73001C52504D001D460000001A
:1062ED001E4A0000005A250000005B52504D005C14
:1062FD00636E74005D780000000000000000023540
:10630D000000004E6F64652041647200008D010035
:10631D00000000000000003F80000000000002357A
:10632D00000000477270204164720000008F010070
:10633D00000000000000003F8000000000000A384F
:10634D0000000054696D6500000000010C0C010097
:10635D00000000000000003F8000000000000A382F
:10636D000000004461746500000000010BFC010099
:10637D00000000000000003F800000000000040845
:10638D0000000154656D7000000000010BD4020087
:10639D00000000000000003F800000000000041815
:1063AD00000001312E385600000000010BEC0200F8
:1063BD000000000000000040000000000000041874
:1063CD00000001332E335600000000010BD80200EF
:1063DD000000000000000040000000000000041854
:1063ED000000013556657874000000010BE00200D5
:1063FD000000000000000040000000000000041834
:10640D000000013234560000000000010BE40200D0
:10641D00000000000000003F800000000000041894
:10642D000000013234566578740000010BE802005B
:10643D00000000000000003F800000000000040686
:10644D000000014920323456000000010BDC02002F
:10645D0000000000000000400000000000000032BD
:10646D00000004466C61736800000000000000002D
:10647D0000000000000000000000000000000032DD
:10648D000000045265626F6F740000000000000090
:0E649D000000000000000000000000000000F1
:0AA83200C19FC127C126C120C1212A
:0664AB008B3F8A4089418D
:1064B1009000011207216438706085424885434984
:1064C10085444AF54B754C0A7B017A0B79F012A58C
:1064D100227B017A0B79F012000EC3EF940AEE646D
:1064E1008094805032E4900C29F07B017A0B79F092
:1064F10012000EC3740A9FFFE49EFE900C29E0C3B4
:106501009FEE6480F8748098500D7F2012AC6D90DE
:106511000C29E004F080D3026772E4900BF0F0AB39
:106521003FAA40A9419000021207216068E4900C43
:1065310029F0900C29E075F005A4245CF582E4347F
:1065410062F583E493FF64636019AB3FAA40A941FC
:10655100900002120721FEEF6E6008900C29E00402
:10656100F080CF900C29E0FF75F005A4245CF58242
:10657100E43462F583E493601CEF75F005A4245DB7
:10658100F9746235F07548FFF549894A7B017A0B48
:1065910079F012A3C7AB3FAA40A9419000011207AD
:1065A100216066E4900C29F0900C29E075F005A4B7
:1065B100248EF582E43462F583E493FF6019AB3FE6
:1065C100AA40A941900001120721FEEF6E600890D8
:1065D1000C29E004F080D1900C29E0FF75F005A4AE
:1065E100248EF582E43462F583E493601CEF75F048
:1065F10005A4248FF9746235F07548FFF549894A7D
:106601007B017A0B79F012A3C77B017A0B79F01227
:10661100000E900C2AEFF0AB3FAA40A941120708E7
:1066210014601D14606424FE70030266DB240460A0
:10663100030267727BFF7A61797D12AAAA026772EF
:10664100AB3FAA40A941900004120721900C2A30C7
:10665100E11CE0FFC3740A9FF548AB42AA43A94479
:10666100120708F5497BFF7A61798802676FE0FFBD
:10667100C3740A9FF548AB42AA43A944120708F51F
:10668100497BFF7A61798E02676FAB3FAA40A941CE
:10669100900004120721900C2A30E11FE0FFC3741F
:1066A1000A9FF548AB42AA43A94412081FF54A853F
:1066B100F0497BFF7A61799402676FE0FFC3740A46
:1066C1009FF548AB42AA43A94412081FF54A85F039
:1066D100497BFF7A61799902676FAB3FAA40A94173
:1066E10090000412072130E033900C2AE0FFC374BC
:1066F1000A9FF548900010120721FF600280027F77
:10670100038F49AB42AA43A9441209218F4D8E4CF4
:106711008D4B8C4A7BFF7A61799E8052AB3FAA40B8
:10672100A941900004120721900C2A30E121E0FFD9
:10673100C3740A9FF548AB42AA43A9441209218FA9
:106741004C8E4B8D4A8C497BFF7A6179A6801FE084
:10675100FFC3740A9FF548AB42AA43A94412092119
:106761008F4C8E4B8D4A8C497BFF7A6179AC124EEE
:0A677100F67B017A0B79F012AAAA58
:01677B0022FB
:0D291500900C1CE0FBA3E0FAA3E0F97DFFAD
:102922008D428B3F8A408941900001120721643811
:102932007003023126AB3FAA40A94112070824FEC8
:102942007003022B8724FE7003022DE02403600330
:1029520002312690000412072120E103022A41AB32
:102962003FAA40A9419000191209CCC000C001C081
:1029720002C003AC42EC1203BBD003D002D001D0A0
:102982000012019EC004C005C006C007900BC6E03D
:10299200FC1203BBD003D002D001D0001200AD1252
:1029A20003EF900BC6EFF0AB3FAA40A94190001590
:1029B2001209419000111209CC1203447003023132
:1029C20026AB3FAA40A941900011120941C004C0A0
:1029D20005C006C007900BC6E0FC1203BBA804A901
:1029E20005AA06AB07D007D006D005D004120344CF
:1029F2005014AB3FAA40A9419000111209411203A1
:102A0200EF900BC6EFF0AB3FAA40A9419000151220
:102A12000941C004C005C006C007900BC6E0FC1205
:102A220003BBA804A905AA06AB07D007D006D005A8
:102A3200D00412034460025003023126022B72E5D5
:102A420042F4704CAB3FAA40A941900011120941D7
:102A5200C004C005C006C007900BC6E0FCE4120328
:102A6200BBA804A905AA06AB07D007D006D005D09B
:102A720004120344701AAB3FAA40A94190001512F8
:102A820009419000111209CC12034460030231265D
:102A9200AB3FAA40A9419000191209CCC000C00165
:102AA200C002C003AC42EC1203BBD003D002D0017F
:102AB200D00012019EC004C005C006C007900BC61C
:102AC200E0FCE41203BBD003D002D001D00012001C
:102AD200AD1203EF900BC6EFF0AB3FAA40A94190B5
:102AE20000151209419000111209CC12034470031F
:102AF200023126AB3FAA40A941900011120941C000
:102B020004C005C006C007900BC6E0FCE41203BB7C
:102B1200A804A905AA06AB07D007D006D005D004A1
:102B22001203445014AB3FAA40A94190001112096C
:102B3200411203EF900BC6EFF0AB3FAA40A94190C0
:102B42000015120941C004C005C006C007900BC69B
:102B5200E0FCE41203BBA804A905AA06AB07D00750
:102B6200D006D005D004120344600250030231267D
:102B7200AB3FAA40A9419000151209411203EF9000
:102B82000BC6EFF022AB3FAA40A941900004120706
:102B92002120E103022C859000191209CCC000C04B
:102BA20001C002C003AC42EC1203BBD003D002D07E
:102BB20001D00012019EC004C005C006C007900BE0
:102BC200C6E0FCA3E0FDEC1203B6D003D002D001B4
:102BD200D0001200AD1203EF900BC6EEF0A3EFF09F
:102BE200AB3FAA40A9419000151209419000111271
:102BF20009CC1203447003023126AB3FAA40A9411B
:102C0200900011120941C004C005C006C007900B14
:102C1200C6E0FCA3E0FDEC1203B6A804A905AA06CF
:102C2200AB07D007D006D005D0041203445017AB2F
:102C32003FAA40A9419000111209411203EF900BE3
:102C4200C6EEF0A3EFF0AB3FAA40A94190001512E7
:102C52000941C004C005C006C007900BC6E0FCA332
:102C6200E0FDEC1203B6A804A905AA06AB07D0073B
:102C7200D006D005D004120344600250030231266C
:102C8200022DC8E542F4704FAB3FAA40A941900023
:102C920011120941C004C005C006C007900BC6E06E
:102CA200FCA3E0FDE41203B6A804A905AA06AB073B
:102CB200D007D006D005D004120344701AAB3FAA45
:102CC20040A9419000151209419000111209CC123D
:102CD20003446003023126AB3FAA40A94190001988
:102CE2001209CCC000C001C002C003AC42EC120306
:102CF200BBD003D002D001D00012019EC004C00597
:102D0200C006C007900BC6E0FCA3E0FDE41203B6C8
:102D1200D003D002D001D0001200AD1203EF900B0D
:102D2200C6EEF0A3EFF0AB3FAA40A9419000151206
:102D320009419000111209CC12034470030231269A
:102D4200AB3FAA40A941900011120941C004C0053D
:102D5200C006C007900BC6E0FCA3E0FDE41203B678
:102D6200A804A905AA06AB07D007D006D005D0044F
:102D72001203445017AB3FAA40A941900011120917
:102D8200411203EF900BC6EEF0A3EFF0AB3FAA4067
:102D9200A941900015120941C004C005C006C00730
:102DA200900BC6E0FCA3E0FDE41203B6A804A9055B
:102DB200AA06AB07D007D006D005D00412034460A0
:102DC200025003023126AB3FAA40A94190001512DE
:102DD20009411203EF900BC6EEF0A3EFF022AB3FD6
:102DE200AA40A94190000412072120E003022EA26A
:102DF200900BC6E0F8A3E0F9A3E0FAA3E0FBC00061
:102E0200C001C002C003AB3FAA40A9419000191201
:102E120009CCC000C001C002C003AC42EC1203BB2B
:102E2200D003D002D001D00012019ED003D002D034
:102E320001D0001200AD900BC6120A08AB3FAA40A7
:102E4200A941900011120941900BC6E0F8A3E0F9E4
:102E5200A3E0FAA3E0FB1203445012AB3FAA40A93D
:102E620041900011120941900BC6120A08AB3FAA09
:102E720040A941900015120941900BC6E0F8A3E069
:102E8200F9A3E0FAA3E0FB1203446002500302310B
:102E920026AB3FAA40A941900015120941023120F8
:102EA200AB3FAA40A94190000412072120E103028E
:102EB2002FBD9000191209CCC000C001C002C0038E
:102EC200AC42EC1203BBD003D002D001D0001201FD
:102ED2009EC004C005C006C007900BC6E0FCA3E07C
:102EE200FDA3E0FEA3E0FFEC1203B1D003D002D0B9
:102EF20001D0001200AD1203EF900BC6120A08AB0C
:102F02003FAA40A9419000151209419000111209EF
:102F1200CC1203447003023126AB3FAA40A9419070
:102F22000011120941C004C005C006C007900BC6BB
:102F3200E0FCA3E0FDA3E0FEA3E0FFEC1203B1A8D6
:102F420004A905AA06AB07D007D006D005D0041203
:102F520003445015AB3FAA40A94190001112094108
:102F62001203EF900BC6120A08AB3FAA40A9419088
:102F72000015120941C004C005C006C007900BC667
:102F8200E0FCA3E0FDA3E0FEA3E0FFEC1203B1A886
:102F920004A905AA06AB07D007D006D005D00412B3
:102FA200034460025003023126AB3FAA40A941907C
:102FB20000151209411203EF023120E542F4705567
:102FC200AB3FAA40A941900011120941C004C005BB
:102FD200C006C007900BC6E0FCA3E0FDA3E0FEA381
:102FE200E0FFE41203B1A804A905AA06AB07D007C3
:102FF200D006D005D004120344701AAB3FAA40A9F0
:10300200419000151209419000111209CC1203449B
:103012006003023126AB3FAA40A941900019120970
:10302200CCC000C001C002C003AC42EC1203BBD052
:1030320003D002D001D00012019EC004C005C00618
:10304200C007900BC6E0FCA3E0FDA3E0FEA3E0FFF7
:10305200E41203B1D003D002D001D0001200AD12AD
:1030620003EF900BC6120A08AB3FAA40A941900099
:10307200151209419000111209CC12034470030287
:103082003126AB3FAA40A941900011120941C00468
:10309200C005C006C007900BC6E0FCA3E0FDA3E09C
:1030A200FEA3E0FFE41203B1A804A905AA06AB0738
:1030B200D007D006D005D0041203445015AB3FAA66
:1030C20040A9419000111209411203EF900BC61260
:1030D2000A08AB3FAA40A941900015120941C00459
:1030E200C005C006C007900BC6E0FCA3E0FDA3E04C
:1030F200FEA3E0FFE41203B1A804A905AA06AB07E8
:10310200D007D006D005D00412034460174015AB97
:103112003FAA40A9419000151209411203EF900BFA
:05312200C6120A08229C
:10A793008F3FE92405F9E43AFA78F07C0B7D017EDA
:10A7A300007F081206E2E4900BF8F0900BF6E0FF4E
:10A7B3006007900BF5F0E4A3F0853F4875490175F8
:10A7C3004A0B754BF07BFF7A6179B2124EF67BFF31
:07A7D3007A6179BA02AAAA1B
:100B9500126A3DEF6003D21F22301F40E4900BD351
:100BA500F0900BCB120A2D00000000900BCF120A1B
:100BB5002D00000000C222C223C224C225E4900CED
:100BC50022F012ACBDE47B2C7A01F9F8C31208FDC2
:100BD500400302166EC21FD214129FA220271EC206
:100BE50014129FA2900C22EFF0700302165ED2271A
:100BF500E06402600302165ED22602165E2026031A
:100C0500020FCC900BFC742DF0E4A3F0900C0C7447
:100C15002DF0E4A3F075420175430C754423754529
:100C250002FB7D02FF128374900C23E0C4F854F09C
:100C3500C868FCA3E0C4540F48FDE41203B6E4FB06
:100C4500FAF978411202A7900C25120A08E4FFFE72
:100C55007D207C41900C25E0F8A3E0F9A3E0FAA300
:100C6500E0FB12019EE4FBFAF9783F1200AD120396
:100C7500EFEC1203B1E4FBFA792078411202A79058
:100C85000BD4120A0875420175430C75442375454A
:100C9500027B017D02E4FF128374900C23E0C4F80B
:100CA50054F0C868FCA3E0C4540F48FDE41203B631
:100CB500E4FBFA79A0784012019EE4FBFA7980788A
:100CC500451202A7900C25120A08E4FFFE7DC87C98
:100CD50042900C25E0F8A3E0F9A3E0FAA3E0FB12AB
:100CE500019EE4FBFAF9783F1200AD1203EFEC1216
:100CF50003B1E4FBFA79C878421202A7900BD81227
:100D05000A0875420175430C7544237545027B023B
:100D15007D02E4FF128374900C23E0C4F854F0C8FC
:100D250068FCA3E0C4540F48FDE41203B6E4FBFAE3
:100D35007920784012019EE4FBFA79807845120209
:100D4500A7900C25120A08900C25E0FCA3E0FDA352
:100D5500E0FEA3E0FF7B007AC0792878451202A760
:100D6500900C25120A08900C25E0FCA3E0FDA3E0F9
:100D7500FEA3E0FF7B007AC0795A784612019E9067
:100D85000C25120A08E4FFFE7DC87C42900C25E084
:100D9500F8A3E0F9A3E0FAA3E0FB12019EE4FBFA55
:100DA500F9783F1200AD1203EFEC1203B1E4FBFA40
:100DB50079C878421202A7900BDC120A0875420125
:100DC50075430C7544237545027B037D02E4FF12D0
:100DD5008374900C23E0C4F854F0C868FCA3E0C405
:100DE500540F48FDE41203B6E4FBFA79C8784012C3
:100DF500019EE4FBFA798078451202A7900C251232
:100E05000A08E4FFFE7DC87C42900C25E0F8A3E0CB
:100E1500F9A3E0FAA3E0FB12019EE4FBFAF9783F9F
:100E25001200AD1203EFEC1203B1E4FBFA79C878B6
:100E3500421202A7900BE0120A0875420175430C95
:100E45007544237545027B047D02E4FF128374908B
:100E55000C23E0C4F854F0C868FEA3E0C4540F485E
:100E6500FF7C007D0B120782AC06AD07E41203B6CA
:100E7500E4FBFA7920784012019EE4FBFA79807848
:100E8500451202A7900C25120A08E4FFFE7DC87CD6
:100E950042900C25E0F8A3E0F9A3E0FAA3E0FB12E9
:100EA500019EE4FBFAF9783F1200AD1203EFEC1254
:100EB50003B1E4FBFA79C878421202A7900BE41259
:100EC5000A0875420175430C7544237545027B0577
:100ED5007D02E4FF128374900C23E0C4F854F0C83B
:100EE50068FEA3E0C4540F48FF7C007D0B12078207
:100EF500AC06AD07E41203B6E4FBFA79207840129C
:100F0500019EE4FBFA798078451202A7900C251220
:100F15000A08E4FFFE7DC87C42900C25E0F8A3E0BA
:100F2500F9A3E0FAA3E0FB12019EE4FBFAF9783F8E
:100F35001200AD1203EFEC1203B1E4FBFA79C878A5
:100F4500421202A7900BE8120A0875420175430C7C
:100F55007544237545027B067D02E4FF1283749078
:100F65000C23E0C4F854F0C868FCA3E0C4540F484F
:100F7500FDE41203B6E4FBFA7920784012019EE401
:100F8500FBFA798078451202A7900C25120A08E42D
:100F9500FFFE7DC87C42900C25E0F8A3E0F9A3E0B4
:100FA500FAA3E0FB12019EE4FBFAF9783F1200ADCB
:100FB5001203EFEC1203B1E4FBFA79C8784212028E
:100FC500A7900BEC120A08900C1C30261374FFF046
:100FD500A37463F0A3740BF0900C20740CF08013D1
:100FE500E51CF0A3E51DF0A3E51EF07882E614905C
:100FF5000C20F0900C20E0FFC394035005E4A3F00F
:10100500801B900BD3E0FE7002800EEE900BD3B5E3
:101015000705E024FE8002E014900C21F07882E6BA
:101025007014202611FDFF12AC837BFF7A6179C312
:10103500124EF6021184E4900C1FF0900C1FE0FD97
:10104500C394034003021184E4FF12AC83900C1F88
:10105500E0FF900C21E02FFFE433FE900BD3E07C02
:1010650000B50708ECB506047F1580027F2012AC99
:101075006D900C1FE0FD7F0112AC83900C1FE0FF0B
:10108500900C21E02FFFE433FE900C20E0FDD3EF20
:101095009D7480F86E98400C7BFF7A6179D8124E6A
:1010A500F602117B900C1FE0FE900C21E0FD2EFF57
:1010B500C007EEFFED2FFFE433FEEF7805C333CE17
:1010C50033CED8F9FF900C1CE0FBA3E0FAA3E02F88
:1010D500F9EA3EFAD00712A793900C1FE0FD7F0AAC
:1010E50012AC83302040900C1FE0FF900C21E02FC4
:1010F500FFE433FE900BD3E07C00B50729ECB50681
:1011050025EF7805C333CE33CED8F9FF900C1CE01C
:10111500FBA3E0FAA3E02FF9EA3EFA754201754315
:101125000B7544C6804D900C1FE0FF900C21E02FFD
:10113500FFE433FEEF7805C333CE33CED8F9FF9005
:101145000C1CE0FBA3E0FAA3E02FF9EA3EFAC0038A
:10115500C002C001900C1CA3E0FAA3E02FF9EA3EFF
:10116500FA90000D120A888B428A438944D001D037
:1011750002D0031264AB900C1FE004F00210409003
:101185000BD3E075F020A430260F240BF9746335DA
:10119500F0FA900C1C74FF800D251EF9E51D35F045
:1011A500FA900C1CE51CF0A3EAF0A3E9F030215AF3
:1011B5007D03E4FF12AC837BFF7A6179EC12AAAA66
:1011C500900BCAE075F003A4240DFF900C21E0FEFE
:1011D500900BD3E0C39EFD12AC8320080A30220792
:1011E500C221E4FF12ACF620090302165E30230388
:1011F50002165E900BCAE004F0E064036003021679
:101205005EC221FF12ACF602165E2020030213D344
:101215007D03E4FF12AC837BFF7A62790112AAAAEF
:10122500900C21E0FF900BD3E0C39FFD7F1312AC20
:101235008320080A302207C220E4FF12ACF63009E9
:1012450053202350C220E4FF12ACF6900C1CE0FBA7
:10125500A3E0FAA3E0F9120708FF7E00900C1CA397
:10126500A3E090000D120A88A801AC02AD037B0132
:101275007A0B79C61206E2302612900BD3E0FF6096
:1012850003B40110D228788076F18008900BD3E062
:10129500FF12AC27300A0F20240C12291512ACBD01
:1012A500900BCB120A08300A2D12ACBDA804A90573
:1012B500AA06AB07900BCBE0FCA3E0FDA3E0FEA3E1
:1012C500E02446FFE43EFEE43DFDE43CFCD3120889
:1012D500FD4003122915300A3B12ACBDA804A9052F
:1012E500AA06AB07900BCBE0FCA3E0FDA3E0FEA3B1
:1012F500E024F4FFEE3401FEE43DFDE43CFCD312B2
:1013050008FD4010900C1CE0FBA3E0FAA3E0F97D7A
:10131500F7122922200A0A900BCB120A2D00000091
:1013250000300B1C202519900C1CE0FBA3E0FAA350
:10133500E0F97D0112292212ACBD900BCF120A08EB
:10134500300B3A12ACBDA804A905AA06AB07900B51
:10135500CFE0FCA3E0FDA3E0FEA3E02446FFE43ECE
:10136500FEE43DFDE43CFCD31208FD4010900C1C4E
:10137500E0FBA3E0FAA3E0F97D01122922300B3B43
:1013850012ACBDA804A905AA06AB07900BCFE0FCDB
:10139500A3E0FDA3E0FEA3E024F4FFEE3401FEE4A8
:1013A5003DFDE43CFCD31208FD4010900C1CE0FB15
:1013B500A3E0FAA3E0F97D09122922300B030216F6
:1013C5005E900BCF120A2D0000000002165E7D0311
:1013D500E4FF12AC837882E6D394005003302637BD
:1013E500900C1CE0FBA3E0FAA3E0F99000191209A8
:1013F50041E4FBFAF9F81203444014900C1CE0FB9D
:10140500A3E0FAA3E0F990000412072130E2087B7B
:10141500FF7A62791680067BFF7A62792312AAAA7F
:101425007F1212AC6D7BFF7A62793012AAAA7F1304
:1014350012AC6D7BFF7A62793612AAAA20080C30AD
:101445002209C227C226D214129FA220090302151F
:101455003C30230302153C7882E6D394004061902A
:101465000C1CE0FBA3E0FAA3E0F9120708FFD394F4
:1014750004504DEF94004048900019120941E4FBD7
:10148500FAF9F81203445038D220900C1CE0FBA363
:10149500E0FAA3E0F9120708FF7E0090000D120A9A
:1014A5008878C67C0B7D011206E2900C21E0FF9046
:1014B5000BD3E0C39FFD7F1312AC837F0112ACF603
:1014C50030262A900BD3E0FF64026004EFB4031DBD
:1014D500D221E4900BCAF0900C21E0FF900BD3E0F1
:1014E500C39FFD7F0D12AC837F0112ACF63026370A
:1014F500900BD3E0640B702FD228788076F112AD73
:1015050015E4FDFF12AC837BFF7A62793812AAAA33
:101515007D01E4FF12AC837BFF7A62794B12AAAAA4
:101525007FB87E0B12AA7F30260D900BD3E0B40C4A
:1015350006E4F58475EF10300A2A202427900BD392
:10154500E070122026077882E614F0800E900BD307
:10155500740CF08006900BD3E014F012ACBD900B28
:10156500CB120A08300A4812ACBDA804A905AA0680
:10157500AB07900BCBE0FCA3E0FDA3E0FEA3E024CA
:1015850046FFE43EFEE43DFDE43CFCD31208FD408D
:101595001E900BD3E070122026077882E614F080A7
:1015A5000E900BD3740CF08006900BD3E014F02052
:1015B5000A0A900BCB120A2D000000003026089075
:1015C5000C1F740DF080077882E6900C1FF0300B2D
:1015D50025202522900BD3E02401FFE433FE900C57
:1015E5001FE0FD7C00120794900BD3EDF012ACBD0B
:1015F500900BCF120A08300B4312ACBDA804A90505
:10160500AA06AB07900BCFE0FCA3E0FDA3E0FEA389
:10161500E02446FFE43EFEE43DFDE43CFCD3120835
:10162500FD4019900BD3E02401FFE433FE900C1F1D
:10163500E0FD7C00120794900BD3EDF0200B0A908F
:101645000BCF120A2D00000000300A0D300B0A20C6
:101655002607E4900BD3F0D226A2089222A2099283
:0916650023A20A9224A20B922593
:01166E002259
:048374008D408B416C
:108378007B08E4FD12AC67E4900C31F0E54054084A
:10838800D394004003D38001C392B30000000000DF
:10839800000000000000000000000000000000D203
:1083A800B000000000000000000000000000000015
:1083B8000000000000C2B0E54025E0F540900C3117
:1083C800E004F0E0B404B5E4900C31F0E541540861
:1083D800D394004003D38001C392B300000000008F
:1083E800000000000000000000000000000000D2B3
:1083F800B0000000000000000000000000000000C5
:108408000000000000C2B0E54125E0F541900C31C4
:10841800E004F0E0B404B5E4900C31F0E54575F003
:1084280008A4FF900C31E0FDC39FE5F06480F87468
:108438008098505CED9400400FE05407700A0425C2
:1084480044F544E43543F543C2B0000000000000A1
:108458000000000000000000000000000000AB4227
:10846800AA43A94412070825E0FFA2B4E4334F1237
:10847800074ED2B00000000000000000000000001D
:108488000000000000000000900C31E004F0808C37
:10849800D2B2000000000000000000000000000050
:0684A800000000000000CE
:0184AE0022AB
:049123007D0AAF45CD
:049127008D468B479F
:10912B00D2B20000000000000000000000000000B0
:10913B00000000000000C2B20000000000000000B0
:10914B000000000000000000000000007B08E4FDB0
:10915B0012AC67E4900C31F0E5465408D394004010
:10916B0003D38001C392B300000000000000000095
:10917B000000000000000000000000D2B000000062
:10918B0000000000000000000000000000000000D4
:10919B0000C2B0E54625E0F546900C31E004F0E066
:1091AB00B404B5E4900C31F0E5475408D394004077
:1091BB0003D38001C392B300000000000000000045
:1091CB000000000000000000000000D2B000000012
:1091DB000000000000000000000000000000000084
:1091EB0000C2B0E54725E0F547900C31E004F0E014
:0391FB00B404B504
:0191FE00224E
:10A66600E4900C20F0EF5480D394004003D3800193
:10A67600C392B300000000000000000000000000CC
:10A6860000000000000000D2B00000000000000042
:10A6960000000000000000000000000000C2B0EF53
:0DA6A60025E0FF900C20E004F0E0B408B8BF
:01A6B3002284
:02939C008F45FB
:10939E00E4FB7D07129127E4FB129123E4FF12A652
:1093AE0066E4FF12A6667B02129123E4FF12A66604
:1093BE00E4FF12A666E4900C1DF0900C1DE0FBC3BA
:1093CE00940750697D0CAF45129127900C1DE0FF5C
:1093DE00700AA37403F0A37420F08017EF900C1E94
:1093EE00B402097401F0A374D9F08007740FF0A3CE
:1093FE0074FFF0900C1EE0C4F854F0C8A3E0C454FF
:10940E000F48FF12A666900C1FE0540FC4F8540FBD
:10941E00C868FF12A666E4FF12A666E4FF12A666EF
:10942E007F3A12A666900C1DE004F0808DE4FB7D61
:10943E000DAF451291277FFF12A6667FFF12A6661B
:0F944E00E4FF12A666E4FF12A6667F1402A6666C
:10AB8300E4FB7D09129127D2B2000000000000000F
:0EAB9300000000000000000000000000002292
:04AAD4008F6B8D6C8B
:10AAD8007B017A0C7947129A1CE56C900C4760064A
:10AAE800E04401F08004E054FEF0900C47E0FDAF34
:04AAF8006B029E91BE
:10AC3F007B017A0C7948E4FF129A1C900C48E030A3
:07AC4F00E7037F00227F01F3
:01AC560022DB
:10ABF5007B017A0C7949E4FF129A1C900C49E030EC
:08AC0500E704540FFF227F0059
:01AC0D002224
:10ABDA007B017A0C794A129A1C900C4AE0FFF460C5
:0AABEA0007EF60047F0180027F0086
:01ABF400223E
:03AD5300202000BD
:0AA89300AB3FAA40A941120721FFC4
:02A89D008F47E3
:10A89F00E478ACF6E5471392927F0A7E0012A36F1D
:10A8AF00D2937F0A7E0012A36FC293E547C313F5BD
:0AA8BF004778AC06E6C3940840DABF
:01A8C900226C
:02A096008F1F1A
:10A09800C293E4F58475D2FF75D30F7F0AFE12A32D
:10A0A8006F75840F43A504AF1F12A89D75840F53C5
:10A0B800A5FBD2927F0A7E0012A36FE47876F61889
:10A0C800F6787776013092077876E6797747F6D290
:10A0D800937F0A7E0012A36FC2937F0A7E0012A3A9
:10A0E8006F7877E625E0F6787506E6C3940840D5DC
:10A0F800E4F584F5D2F5D37F0AFE12A36F7876E6ED
:01A10800FF57
:01A109002233
:0691FF008B3F8A4089410C
:10920500C293E4F58475D2FF75D30F7F0AFE12A3CE
:109215006F75840F43A5047FBF12A89D75840F53F6
:10922500A5FBD2927F0A7E0012A36FE478A9F6E42B
:1092350078AAF678A8F678AB760130920778AAE690
:1092450079AB47F6D2937F0A7E0012A36FC2937F54
:109255000A7E0012A36F78ABE625E0F678A806E64D
:10926500C3940840D578A9E6FFC39403501908E6CE
:10927500FEEFFDC374059DFDE49400AB3FAA40A934
:10928500418D82F583801E78A9E6FFC394055018A9
:1092950008E6FEEF7C0024FDF582EC34FFF583AB98
:1092A5003FAA40A941EE801178A9E6B4060E08E66A
:1092B500AB3FAA40A94190000212076078A906E6D3
:1092C500C394075003029234E4F584F5D2F5D37FB5
:0592D5000AFE02A36F78
:10A96C008F458D46C293E4F58475D2FF75D30F7F66
:10A97C000AFE12A36F75840F43A504AF4512A89D60
:10A98C00AF4612A89DE4F584F5D2F5D37F0AFE02FA
:02A99C00A36FA7
:10A020008B3F8A408941C293E4F58475D2FF75D392
:10A030000F7F0AFE12A36F75840F43A5047FBE1223
:10A04000A89D90000512A89390000412A893AB3F1E
:10A05000AA40A94190000312A899AB3FAA40A94188
:10A06000120708FF12A89DAB3FAA40A9419000012A
:10A0700012A8997F0112A89DAB3FAA40A941900068
:10A080000212A899E4FF12A89DE4F584F5D2F5D355
:06A090007F0AFE02A36F2F
:10A857008D6FEF14601614601914601C14601F14B8
:10A86700602224057025AD6F7F86801CAD6F7F88C1
:10A877008016AD6F7F8C8010AD6F7F84800AAD6FBF
:0CA887007F828004AD6F7F8012A96C22DC
:108B88008B088A09890A120708FFF47049AB0BAAF7
:108B98000CA90D900007743F120760900006743FFF
:108BA800120760900004743F120760900003743F3E
:108BB800120760900001743F120760743F12074E5D
:108BC800AB0BAA0CA90D900005742D12076090003C
:108BD80002742D028C85EFC4540F2430AB0BAA0C01
:108BE800A90D12074EAB08AA09A90A120708540FC3
:108BF8002430AB0BAA0CA90D90000112076090005D
:108C080002742D120760AB08AA09A90A9000011284
:108C18000721C4540F2430AB0BAA0CA90D900003F4
:108C2800120760AB08AA09A90A900001120721548B
:108C38000F2430AB0BAA0CA90D900004120760900A
:108C48000005742D120760AB08AA09A90A90000252
:108C5800120721C4540F2430AB0BAA0CA90D9000A5
:108C680006120760AB08AA09A90A90000212072198
:108C7800540F2430AB0BAA0CA90D90000712076003
:088C8800900008E412076022CD
:108963008B0E8A0F8910120708F47049AB11AA12F3
:10897300A913900007743F120760900006743F121A
:108983000760900004743F120760900003743F1265
:108993000760900001743F120760743F12074EABEB
:1089A30011AA12A913900005743A120760900002ED
:1089B300743A028A6DAB0EAA0FA910900003120736
:1089C30021C4540F2430AB11AA12A91312074EABC2
:1089D3000EAA0FA910900003120721540F2430ABE5
:1089E30011AA12A913900001120760900002743AB1
:1089F300120760AB0EAA0FA910900004120721C43E
:108A0300540F2430AB11AA12A9139000031207606C
:108A1300AB0EAA0FA910900004120721540F2430A3
:108A2300AB11AA12A91390000412076090000574F9
:108A33003A120760AB0EAA0FA91090000512072186
:108A4300C4540F2430AB11AA12A9139000061207C5
:108A530060AB0EAA0FA910900005120721540F2432
:108A630030AB11AA12A913900007120760900008F7
:058A7300E4120760227F
:10A616007B017A0C79341291FF900C34E0F4603FA0
:10A62600750B01750C0C750D3A7B017A0C79341299
:10A636008B887B017A0C793A12AAAA7BFF7AAD79CC
:10A646005312AAAA75110175120C75133A7B017A79
:0FA656000C79341289637B017A0C793A12AAAA23
:01A6650022D2
:10AC9700E4FF12A0967879EFF6F460047F01800252
:02ACA7007F002C
:01ACA9002288
:07AD3B00E4FD7F8E02A96C0C
:1038AC004C45442D4465627567004C45442D50755C
:1038BC006C7365720044696E203556004F70744904
:1038CC006E0043504C4400446F75742035562F32B3
:1038DC0034560052656C616973004F70744F757487
:1038EC000055696E20302D322E35560055696E20EC
:1038FC002B2D3130560049696E20302D322E356D0E
:10390C00410049696E20302D32356D410055696E8C
:10391C0020302D322E3556204673740055696E209A
:10392C002B2D31305620466173740049696E20305E
:10393C002D322E356D41204673740049696E20304E
:10394C002D32356D41204673740055696E202B2D38
:10395C0031305620446966660055696E202B2D3136
:10396C00305620466C740043696E20302D31306E19
:10397C00460043696E20302D31754600505431306D
:10398C00302D38005054313030302D380041443512
:10399C0039300050543130302D32005054313030E9
:1039AC00302D32004345524E4F582D3200554F7535
:1039BC007420302D322E355600554F7574202B2D1A
:1039CC0031305600494F757420302D322E356D41F3
:1039DC0000494F757420302D32356D41004C6971A2
:1039EC002E4865206C6576656C00554F75742032D9
:1039FC0030305600245265763A2034313639202442
:103A0C0000013400000050254F75740000000100C7
:103A1C00010000000000437F00003F800000000018
:103A2C00000418000001502555696E2300000100A8
:103A3C00080400000000000000000000000000006E
:103A4C00000418000001502555696E230000010088
:103A5C000404000000000000000000000000000052
:103A6C00000418000001502555696E230000010068
:103A7C000204000000000000000000000000000034
:103A8C00000418000001502555696E230000010048
:103A9C00080400000000000000000000000000000E
:103AAC00000134000008502552616E67650001006A
:103ABC0000000000000000000000000000000000FA
:103ACC000004180000015025556F75742300010087
:103ADC00080200000000402000003DCCCCCD0000CE
:103AEC000004180000015025556F75742300010067
:103AFC000802C1200000412000003F00000000002F
:103B0C00000406FD0001502549696E2300000100E8
:103B1C00080400000000000000000000000000008D
:103B2C0000041DF70001502543696E2300000100BD
:103B3C000404000000000000000000000000000071
:103B4C00000408000001502554230000000001006F
:103B5C00080200000000000000000000000000004F
:103B6C00000406FD000950254578636974000100C6
:103B7C000001000000000000000000000000000038
:103B8C00000408000001502554230000000001002F
:103B9C00080200000000000000000000000000000F
:103BAC00000408000001502554230000000001000F
:103BBC0002020000000000000000000000000000F5
:103BCC0000040700000150255423000000000100F0
:103BDC0002020000000000000000000000000000D5
:103BEC00000406FD00015025496F75742300010087
:103BFC0008020000000041A000003DCCCCCD00002C
:103C0C00000406FD00095025457863697400010025
:103C1C0000010000000042C800003F8000000000CE
:103C2C0000045A00000950254C4F66730000010037
:103C3C000002000000000000000000000000000076
:103C4C0000045D00000950254C4761696E000100BD
:103C5C000002000000000000000000000000000056
:103C6C000002030000085025546F66660000010036
:103C7C000000000000000000000000000000000038
:103C8C000002030000085025546F6E000000010074
:103C9C000000000000000000000000000000000018
:103CAC0000045A00000150254C696E000000010010
:103CBC0000010000000000000000000000000000F7
:103CCC00000132000000502544696E230000010001
:103CDC0008010000000000000000000000000000CF
:103CEC00000132000000502544696E2300000100E1
:103CFC0004010000000000000000000000000000B3
:103D0C000001320000005025446F7574230001003F
:103D1C000801000000003F8000003F800000000010
:103D2C00000132000000502552656C230000010098
:103D3C000401000000003F8000003F8000000000F4
:103D4C0000013200000050254F7574230000010063
:103D5C000401000000003F8000003F8000000000D4
:103D6C0000041800000150255544230000000100F8
:103D7C00080300000000434800003F8000000000E2
:103D8C00000418000001502555230000000001001C
:103D9C00080300000000000000000000000000000C
:103DAC00000406FA00015025492300000000010020
:103DBC0008030000000000000000000000000000EC
:103DCC000001FF38ACFF3A0D01FFA31702FF38B614
:103DDC000000000100000020FF38C1FF3CCD01FFB6
:103DEC008A7821FF38C8FF3CED01FF8A7822FF3822
:103DFC00CEFF3CCD01FF8A7840FF38D3FF3D0D014B
:103E0C00FF7CA341FF38DFFF3D2D01FF7CA342FF68
:103E1C0038E6FF3D4D01FF7CA360FF38EDFF3A2DE6
:103E2C0001FF56E661FF38F8FF3A2D01FF56E662B6
:103E3C00FF3902FF3B0D01FF56E663FF390EFF3BD6
:103E4C000D01FF56E664FF3919FF3A2D01FF5AC1E7
:103E5C0065FF3928FF3A2D01FF5AC166FF3937FF3C
:103E6C003B0D01FF5AC167FF3947FF3B0D01FF5A5C
:103E7C00C168FF3956FF3A4D01FF56E669FF3965B7
:103E8C00FF3A6D01FF6F9C70FF3973FF3B2D01FFF3
:103E9C006CF071FF397EFF3B2D01FF6CF072FF3926
:103EAC0088FF3B4D02FF49E173FF3990FF3B4D0208
:103EBC00FF49E174FF3999FF3B8D01FF677C75FF6A
:103ECC00399FFF3BAD01FF44C976FF39A7FF3BADDE
:103EDC0001FF44C977FF39B0FF3BCD01FF44C980D6
:103EEC00FF39B9FF3ACD01FF748381FF39C5FF3A21
:103EFC00ED01FF3F6882FF39D0FF3BED01FF74837A
:103F0C0083FF39DDFF3BED01FF748384FF39E9FF4B
:103F1C003C0D06FF166F85FF39F6FF3D6D03FF3133
:103F2C002700000000000000000000003CA3D70A9E
:103F3C003D23D70A3DA3D70A3E23D70A3EA3D70A6F
:103F4C003F23D70A3FA3D70A4023D70A050403020D
:0C3F5C000100060706020703000405012F
:06A83C00041400000000FE
:107B2600E5702412F8E6FFE5702413F8E6FD7550BB
:037B3600017B06CA
:107B3900D2B1C2B0C2B2E4900C33F0900C33E0FE83
:107B4900C39404504CEFC8EEC8088002C333D8FC74
:107B59005408D394004003D38001C392B3000000BA
:107B6900000000000000000000000000000000000C
:107B790000D2B0000000000000000000000000007A
:107B890000000000000000C2B0900C33E004F08057
:107B9900AAE4900C33F0900C33E0FFC39403504CEB
:107BA900EDC8EFC8088002C333D8FC5404D394004D
:107BB9004003D38001C392B300000000000000001D
:107BC900000000000000000000000000D2B000002A
:107BD900000000000000000000000000000000009C
:107BE9000000C2B0900C33E004F080AAE4900C339A
:107BF900F0900C33E0FFC39404504CEBC8EFC80875
:107C09008002C333D8FC5408D394004003D38001C5
:107C1900C392B30000000000000000000000000053
:107C290000000000000000D2B000000000000000C9
:107C390000000000000000000000000000C2B09039
:107C49000C33E004F080AAD2B2000000000000006A
:107C590000000000000000000000000000D2B00099
:107C6900000000000000000000000000000000000B
:107C7900000000C2B0C2B2C2B3E55024FF92B0D234
:107C8900B2C2B100000000000000000000000000C6
:097C990000000000000000C2B26E
:017CA20022BF
:10AC5700E5702409F8E6FFE570240AF8E6FD7B06AF
:06AC6700E4F550027B3908
:059C6100F8E6FD7BFFA9
:039C6600CCEBCC78
:109C69007B0312AC67E4900C1CF0EC5480D3940095
:109C79004003D38001C392B300000000000000003C
:109C8900000000000000000000000000D2B0000049
:109C990000000000000000000000000000000000BB
:109CA9000000C2B0EC25E0FC900C1CE004F0E0B42C
:109CB90008B8C2B3D2B200000000000000000000E2
:109CC90000000000000000000000D2B00000000009
:109CD900000000000000000000000000000000007B
:049CE900C2B0C2B291
:019CED002254
:1095C200E5702405F8EFF6E5702412F8E6FFE57081
:0C95D2002413F8E6FDE5702405F8E6FB24
:0395DE00CCEBCC07
:1095E1007B0212AC67E4900C1CF0EC5480D3940025
:1095F1004003D38001C392B30000000000000000CB
:10960100000000000000000000000000D2B00000D7
:109611000000000000000000000000000000000049
:109621000000C2B0EC25E0FC900C1CE004F0E0B4BA
:1096310008B8C2B3D2B20000000000000000000070
:1096410000000000000000000000D2B00000000097
:109651000000000000000000000000000000000009
:04966100C2B0C2B21F
:0196650022E2
:0C97AD00F8E6FD7B00E5702408F97A0066
:0697B9008B448A4589463D
:1097BF00E4FB12AC67D2B200000000000000000012
:1097CF000000000000000000000000D2B000000008
:1097DF00000000000000000000000000000000007A
:1097EF0000C2B0C2B2E4900C1CF0000000000000F8
:1097FF000000000000000000000000000000D2B0D8
:10980F000000000000000000000000000000000049
:10981F0000000000C2B0900C1DE025E0FFA2B4E4F0
:10982F00334FF0900C1CE004F0E0B408BD900C1D19
:0A983F00E0AB44AA45A94602074E1B
:069BD1008B448A45894621
:109BD7007B0112AC67D2B200000000000000000059
:109BE7000000000000000000000000D2B0000000EC
:109BF700000000000000000000000000000000005E
:109C070000C2B0C2B2E4900C1CF0000000000000DB
:109C17000000000000000000000000000000D2B0BB
:109C2700000000000000000000000000000000002D
:109C370000000000C2B0900C1DE025E0FFA2B4E4D4
:109C4700334FF0900C1CE004F0E0B408BD900C1DFD
:0A9C5700E0AB44AA45A94602074EFF
:039E9100CCEDCC49
:109E94007B05E4FD12AC67E4900C4BF0EC5480D3EA
:109EA40094004003D38001C392B30000000000007B
:109EB4000000000000000000000000000000D2B01C
:109EC400000000000000000000000000000000008E
:109ED40000000000C2B0EC25E0FC900C4BE004F064
:109EE400E0B408B8C2B3D2B2000000000000000021
:109EF400000000000000000000000000D2B00000DC
:109F0400000000000000000000000000000000004D
:069F14000000C2B0C2B261
:019F1A002224
:069A1C008B3F8A408941E6
:109A22007B04E4FD12AC67D2B2000000000000002B
:109A320000000000000000000000000000D2B000A2
:109A42000000000000000000000000000000000014
:109A5200000000C2B0C2B2E4900C31F0000000007D
:109A620000000000000000000000000000000000F4
:109A7200D2B0000000000000000000000000000062
:109A8200000000000000C2B0900C32E025E0FFA20E
:109A9200B4E4334FF0900C31E004F0E0B408BD9030
:0C9AA2000C32E0AB3FAA40A94102074E85
:10AC0E007B017A0C791A128233900C1AE0D39400DD
:08AC1E0040047F0180027F0069
:01AC2600220B
:068233008B448A458946D8
:108239007B0712AC67D2B300000000000000000009
:108249000000000000000000000000D2B0000000A3
:108259000000000000000000000000000000000015
:1082690000C2B0D2B300000000000000000000000E
:10827900000000000000000000D2B0000000000073
:10828900000000000000000000000000000000C223
:10829900B0C2B300000000000000000000000000B0
:1082A90000000000000000D2B00000000000000043
:1082B90000000000000000000000000000C2B0E45F
:1082C900900C1BF0C2B30000000000000000000089
:1082D90000000000000000000000D2B00000000013
:1082E9000000000000000000000000000000000085
:1082F900C2B0900C1BE004F0E0B406C830B409AB7E
:1083090044AA45A946E4805FE4900C1BF0000000F4
:108319000000000000000000000000000000000054
:1083290000D2B000000000000000000000000000C2
:1083390000000000000000C2B0900C1DE025E0FF25
:10834900900C1CE033FEA2B4E433FDEF4DFFEEF0D8
:10835900A3EFF0900C1BE004F0E0B410B0900C1CFB
:0A836900E0AB44AA45A94612074EF6
:0183730022E7
:10A8CA00900C17EFF0A3EDF0A3EBF012AC0EEF70C3
:10A8DA0002FF22900C17E0FFA3E0FD7B017A0C79BE
:10A8EA0016128233900C19E0FF900C16E06F700478
:06A8FA007F0180027F00D7
:01A900002234
:03723E00CCEBCCCA
:107241007B0712AC67D2B300000000000000000011
:107251000000000000000000000000D2B0000000AB
:10726100000000000000000000000000000000001D
:1072710000C2B0C2B3000000000000000000000026
:10728100000000000000000000D2B000000000007B
:10729100000000000000000000000000000000C22B
:1072A100B0C2B300000000000000000000000000B8
:1072B10000000000000000D2B0000000000000004B
:1072C10000000000000000000000000000C2B0E467
:1072D100900C44F0D2B30000000000000000000058
:1072E10000000000000000000000D2B0000000001B
:1072F100000000000000000000000000000000008D
:10730100C2B0900C44E004F0E0B406C8D2B2000070
:10731100000000000000000000000000000000006C
:107321000000C2B2D2B30000000000000000000063
:1073310000000000000000000000D2B000000000CA
:10734100000000000000000000000000000000003C
:10735100C2B0C2B300000000000000000000000045
:107361000000000000000000D2B00000000000009A
:107371000000000000000000000000000000C2B09A
:10738100D2B3000000000000000000000000000077
:10739100000000000000D2B000000000000000006A
:1073A100000000000000000000000000C2B0E490F6
:1073B1000C44F0C2B3000000000000000000000017
:1073C100000000000000000000D2B000000000003A
:1073D100000000000000000000000000000000C2EA
:1073E100B0900C44E004F0E0B406C8E4900C44F022
:1073F100EC5480D394004003D38001C392B30000C6
:10740100000000000000000000000000000000007B
:107411000000D2B0000000000000000000000000E9
:107421000000000000000000C2B0EC25E0FC900C60
:1074310044E004F0E0B410B8D2B200000000000053
:107441000000000000000000000000000000C2B2C7
:0A745100E4900C45F0A3F020B427EE
:0D745B00756D01756E0300D56EFCD56DF6E4
:10746800900C46E004F07006900C45E004F0900C97
:0A74780045E0B427DBA3E0B410D612
:0174820022E7
:107CA3001570A870EBF61570A870EDF61570A87036
:047CB300EFF6157063
:107CB700A8700808E664016003027D45E5702404A6
:107CC700F8E6FEE5702403F8E6FF75F008A42EF544
:107CD70082E435F0F583E5822418F582E5833400E4
:107CE700F583E4F0F584E5EF20E119E5702404F865
:107CF700E6FDEF75F008A42D2418F9E43400FA7BAB
:107D070001129BD1E5702403F8E6FFE5702404F81F
:107D1700E6FD75F008EFA42DF582E435F0F583E56F
:107D2700822418F582E5833400F583E0FB1295DEA3
:107D3700E5702403F8E6FFE5702404129C61A8703F
:107D47000808E664026003027E0EE5702406F8CB9D
:107D5700E6CB08E6FA08E6F9120708A870F6603ECF
:107D6700E5702404F8E6FFE5702403F8E675F008EB
:107D7700A42FF582E435F0F583E5822418F582E532
:107D8700833400F583E0FFE5702405F8E6FE74010F
:107D9700C8EEC8088002C333D8FC4FF0803DE570B9
:107DA7002404F8E6FFE5702403F8E675F008A42F2D
:107DB700F582E435F0F583E5822418F582E583340E
:107DC70000F583E0FFE5702405F8E6FE7401C8EED0
:107DD700C8088002C333D8FCF45FF0E5702403F8C9
:107DE700E6FFE5702404F8E6FD75F008EFA42DF52D
:107DF70082E435F0F583E5822418F582E5833400C3
:097E0700F583E0FB1295DE7F001B
:077E1000E5702409F5702262
:108A78001570A870EBF61570A870EDF61570A87053
:048A8800EFF6157080
:108A8C00A8700808E664036003028B7FE570240677
:108A9C00F8CBE6CB08E6FA08E6F9120708603EE5E3
:108AAC00702404F8E6FFE5702403F8E675F008A4DA
:108ABC002FF582E435F0F583E5822418F582E58301
:108ACC003400F583E0FFE5702405F8E6FE7401C878
:108ADC00EEC8088002C333D8FC4FF0803DE570240B
:108AEC0004F8E6FFE5702403F8E675F008A42FF50A
:108AFC0082E435F0F583E5822418F582E5833400B1
:108B0C00F583E0FFE5702405F8E6FE7401C8EEC8B5
:108B1C00088002C333D8FCF45FF0E5702403F8E658
:108B2C00FFE5702404F8E6FD7B00A9707A0012972B
:108B3C00B9E5702405F974017E00C8E7C808800502
:108B4C00C333CE33CED8F9FFA870E6FDEF5DD394D6
:108B5C00007480948040047F0180027F00E57024C3
:108B6C0006F8CBE6CB08E6FA08E6F9EF12074E7FDB
:058B7C000180027F00F2
:078B8100E5702409F57022E4
:10A317001570A870EBF61570A870EDF61570A8709B
:10A32700EFF6A87008E6B4010DA8700808E6FFE587
:10A33700702403129C61A87008E6B40222A8700872
:10A3470008E6FFE5702403F8E6FDE5702405F8CB81
:10A35700E6CB08E6FA08E6F9120708FB1295DE7F56
:08A3670000E5702408F57022E6
:107483001570A870EBF61570A870EDF61570A8705E
:08749300EFF6E57024F9F57035
:10749B002408F8E664026003027642E570240CF8D7
:1074AB00CBE6CB08E6FA08E6F9120921A870120917
:1074BB00FCE5702407F8E6B40209E4FBFA79C87816
:1074CB00428022E5702407F8E6B48209E4FBFA79DE
:1074DB002078408010E5702407F8E6B4832DE4FB98
:1074EB00FA79C87841E8C0E0A87012098BD0E0F8AF
:1074FB001202A77B007AFF797F784712019E120355
:10750B00EFE5702404F8EEF608EFF612AC57E570D1
:10751B002406F8E4F6E5702406F8E6FFC39404505D
:10752B003FEF94014003D38001C392B300000000EE
:10753B000000000000000000000000000000000040
:10754B00D2B00000000000000000000000000000AE
:10755B00000000000000C2B0E5702406F80680B5FC
:10756B00E5702406F8E4F6E5702406F8E6C3940407
:10757B005051E570240BF8E6FF5408D394004003F8
:10758B00D38001C392B30000000000000000000094
:10759B0000000000000000000000D2B0000000005E
:1075AB0000000000000000000000000000000000D0
:1075BB00C2B0E570240BF8EF25E0F6E5702406F871
:1075CB000680A4E5702406F8E4F6E5702406F8E6D8
:1075DB00C394105060E5702404F8E6FE08E6FFEE55
:1075EB005480FCD3E49400EC94004003D38001C39B
:1075FB0092B300000000000000000000000000003B
:10760B00000000000000D2B00000000000000000ED
:10761B00000000000000000000000000C2B0E57098
:10762B002404F8EF25E0FFEE33F608EFF6E57024BF
:09763B0006F8068095D2B17F002B
:07764400E570240FF5702230
:103F68001570A870EBF61570A870EDF61570A870AE
:083F7800EFF6E57024F9F57085
:103F8000E5702408F8E6640260030244C0E570248A
:103F90000CF8CBE6CB08E6FA08E6F9120921A8707E
:103FA0001209FCE4FFFE7D207C41A8701209A312D7
:103FB0000344600B4009A870120A1441200000E479
:103FC000FFFE7D207CC1A8701209A3120344500992
:103FD000A870120A14C1200000E4FFFE7D207C417D
:103FE000A8701209A31200ADE4FBFA79A07841127F
:103FF00002A77B007AFF797F784712019EE4FBFAE3
:10400000F9783F1200AD1203EFE5702404F8EEF6E4
:1040100008EFF612AC57C2B3000000000000000029
:10402000000000000000000000000000D2B000000E
:104030000000000000000000000000000000000080
:104040000000C2B0C2B30000000000000000000089
:1040500000000000000000000000D2B000000000DE
:104060000000000000000000000000000000000050
:10407000C2B0E570240BF8E6FFC394045049E57024
:104080002406F8E4F6E5702406F8E6C39416400327
:1040900002426A0000000000000000000000000072
:1040A00000000000000000D2B0000000000000008E
:1040B00000000000000000000000000000C2B0E5A9
:1040C000702406F80680BEC2B300000000000000A5
:1040D00000000000000000000000000000D2B0005E
:1040E00000000000000000000000000000000000D0
:1040F000000000C2B0D2B3000000000000000000C9
:104100000000000000000000000000D2B00000002D
:10411000000000000000000000000000000000009F
:1041200000C2B0C2B30000000000000000000000A8
:10413000000000000000000000D2B00000000000FD
:10414000000000000000000000000000000000C2AD
:10415000B0C2B3000000000000000000000000003A
:1041600000000000000000D2B000000000000000CD
:1041700000000000000000000000000000C2B0EFDE
:104180005402D394004003D38001C392B3000000D3
:10419000000000000000000000000000000000001F
:1041A00000D2B0000000000000000000000000008D
:1041B00000000000000000C2B0E570240BF8E654D7
:1041C00001D394004003D38001C392B300000000E8
:1041D00000000000000000000000000000000000DF
:1041E000D2B000000000000000000000000000004D
:1041F000000000000000C2B0E5702406F8E4F6E517
:10420000702406F8E6C394105060E5702404F8E6C4
:10421000FE08E6FFEE5480FCD3E49400EC940040EA
:1042200003D38001C392B30000000000000000002F
:104230000000000000000000000000D2B0000000FC
:10424000000000000000000000000000000000006E
:1042500000C2B0E5702404F8EF25E0FFEE33F60865
:10426000EFF6E5702406F8068095C2B30000000062
:10427000000000000000000000000000000000003E
:10428000D2B00000000000000000000000000000AC
:10429000000000000000C2B0C2B300000000000037
:1042A0000000000000000000000000000000D2B08C
:1042B00000000000000000000000000000000000FE
:1042C00000000000C2B0E570240BF8E6FFD39403B1
:1042D0004049E5702406F8E4F6E5702406F8E6C3E4
:1042E000941640030244BE000000000000000000DD
:1042F0000000000000000000000000D2B00000003C
:1043000000000000000000000000000000000000AD
:1043100000C2B0E5702406F80680BEC2B3000000FB
:10432000000000000000000000000000000000008D
:1043300000D2B000000000000000000000000000FB
:1043400000000000000000C2B0D2B3000000000076
:10435000000000000000000000000000000000D28B
:10436000B00000000000000000000000000000009D
:104370000000000000C2B0C2B30000000000000056
:1043800000000000000000000000000000D2B000AB
:10439000000000000000000000000000000000001D
:1043A000000000C2B0C2B300000000000000000026
:1043B0000000000000000000000000D2B00000007B
:1043C00000000000000000000000000000000000ED
:1043D00000C2B0EF5402D394004003D38001C392D3
:1043E000B30000000000000000000000000000001A
:1043F0000000000000D2B00000000000000000003B
:104400000000000000000000000000C2B0E57024C1
:104410000BF8E65401D394004003D38001C392B358
:10442000000000000000000000000000000000008C
:1044300000000000D2B000000000000000000000FA
:1044400000000000000000000000C2B0E57024067B
:10445000F8E4F6E5702406F8E6C394105060E570C1
:104460002404F8E6FE08E6FFEE5480FCD3E4940052
:10447000EC94004003D38001C392B300000000001D
:10448000000000000000000000000000000000D25A
:10449000B00000000000000000000000000000006C
:1044A0000000000000C2B0E5702404F8EF25E0FF32
:1044B000EE33F608EFF6E5702406F8068095D2B1E3
:0244C0007F007B
:0744C200E570240FF57022E4
:0B7F7D007D527F03127F887D037F018F
:107F88001570A870EDF61570A870EFF615701570DD
:107F9800C2B3C2B1000000000000000000000000F1
:107FA8000000000000000000A870E4F6A870E6C316
:107FB80094045031C2B0C2B30000000000000000B9
:107FC800000000000000000000000000D2B0000027
:107FD8000000000000000000000000000000000099
:107FE80000000680C7A870E4F6A870087608A87094
:107FF800E6C39404504AC2B008E6FFA870080856C1
:1080080094004003D38001C392B300000000000035
:108018000000000000000000000000000000D2B0D6
:108028000000000000000000000000000000000048
:1080380000000000A87008EFC313F6A8700680AE11
:10804800D2B20000000000000000000000000000A4
:10805800000000000000C2B2A870E4F6A87008761C
:1080680080A870E6C39408504DC2B008E6FFE570DA
:108078002403F8E65FD394004003D38001C392B38E
:1080880000000000000000000000000000000000E8
:1080980000000000D2B00000000000000000000056
:1080A80000000000000000000000A87008EFC313E3
:1080B800F6A8700680ABD2B1C2B300000000000081
:0E80C8000000000000000000000000000000AA
:0780D600E5702404F570229F
:0A9849001570A870EFF61570157089
:10985300C2B3C2B10000000000000000000000001D
:109863000000000000000000A870E4F6A87008766D
:1098730080A870E6C39408504AC2B008E6FFA870F7
:1098830008085694004003D38001C392B30000003C
:1098930000000000000000000000000000000000C5
:1098A30000D2B00000000000000000000000000033
:1098B30000000000000000A87008EFC313F6A870B2
:1098C3000680AED2B1C2B300000000000000000069
:0B98D30000000000000000000000008A
:0798DE000570057005702202
:0B764B007B00E5702409F97A007F0441
:10765600157015701570A870C6EBC608C6EAC60880
:0D766600C6E9C61570A870EFF61570157016
:10767300C2B1000000000000000000000000000094
:10768300000000000000A870E4F6A870E6FFC394B1
:1076930004503BC2B0EFB40103D38001C392B300E3
:1076A30000000000000000000000000000000000D7
:1076B300000000D2B0000000000000000000000045
:1076C300000000000000000000A8700680BCA87045
:1076D300E4F6A870087608A870E6C39404504AC27A
:1076E300B008E6FFA87008085694004003D3800151
:1076F300C392B3000000000000000000000000007F
:1077030000000000000000D2B000000000000000F4
:1077130000000000000000000000000000A8700846
:10772300EFC313F6A8700680AED2B20000000000CB
:10773300000000000000000000000000000000C284
:10774300B2A870E4F6E5702403F8CBE6CB08E6FABA
:1077530008E6F9120A5E00000000A870E6C3941858
:107763005070C2B0000000000000000000000000E4
:107773000000000000000000E5702403F8CBE6CB16
:1077830008E6FA08E6F9120921780112090EC8EC95
:10779300C8C9EDC9CAEECACBEFCBA2B4E4334BFFE1
:1077A300EAFEE9FDE8FCE5702403F8CBE6CB08E646
:1077B300FA08E6F9120971D2B000000000000000D7
:1077C30000000000000000000000000000A8700698
:1077D3008088D2B10000000000000000000000001B
:0877E30000000000000000009E
:0777EB00E5702406F5702291
:1056E6001570A870EBF61570A870EDF61570A87019
:0856F600EFF6E57024F5F570F4
:1056FE00240CF8E6640160030257C1E570240DF82E
:0C570E00E6FFE570240E127B31127F7D57
:10571A00E5702409F87664E5702409F8E6D3940064
:10572A004023E570240AF87603E570240AF8E6D3E4
:10573A009400400900E570240AF81680ECE570240C
:05574A0009F81680D2F1
:10574F00E570240EF8E6FFE570240DF8E6FE75F01F
:10575F0008A42FF582E435F0F583E5822478F582ED
:10576F00E5833403F5837407F075F008EEA42FF585
:10577F0082E435F0F583E5822478F582E5833403FE
:10578F00F583E04408FD7F02127F88E570240EF850
:10579F00E6FFE570240DF8E675F008A42FF582E416
:1057AF0035F0F583E5822448F582E5833406F583E9
:1057BF00E4F0E570240CF8E6FF64027042E5702413
:1057CF000FF8E6B40839E5702410F8CBE6CB08E6FD
:1057DF00FA08E6F9120708FEE570240EF8E6FDE573
:1057EF0070240DF8E675F008A42DF582E435F0F578
:1057FF0083E5822478F582E5833403F583EEF0EFB9
:10580F0064036003025AB8E570240FF8E6D39407D7
:10581F0040057F00025ABAE570240DF8E6FFE570E7
:10582F00240E1297ADE5702408F8E65401D39400C6
:10583F0040057F00025ABAE570240EF8E6FDE570C8
:10584F00240DF8E6FE75F008A42DF582E435F0F589
:10585F0083E5822448F582E5833406F583E0FFE58E
:10586F0070240FF8E66F60057F00025ABACFEECFB3
:10587F00127B347B00E5702404127651E570240B03
:10588F00F8E66468702CE570240EF8E6FFE57024E6
:10589F000DF8E6FE75F008A42FF582E435F0F583D8
:1058AF00E5822448F582E5833406F583E00454034A
:1058BF00802AE570240EF8E6FFE570240DF8E6FE69
:1058CF0075F008A42FF582E435F0F583E5822448BE
:1058DF00F582E5833406F583E0045407FD75F0087F
:1058EF00EEA42FF582E435F0F583E5822448F582A6
:1058FF00E5833406F583EDF0E570240EF8E6FFE559
:10590F0070240DF8E6FE75F008A42FF582E435F04B
:10591F00F583E5822448F582E5833406F583E0C4F8
:10592F0054F04408FD75F008EEA42FF582E435F02D
:10593F00F583E5822478F582E5833403F583E04D22
:10594F00FD7F02127F88E5702404F812098BE412A0
:10595F0003B1E4FBFA7980784B1202A7E570240EAD
:10596F00F8E6FBE570240DF8E675F008A42BF58238
:10597F00E435F0F583E5822478F582E5833403F589
:10598F0083E025E025E02438F582E4343FF58312E7
:10599F0009BC12019EA8701209FCE570240BF8E6F1
:1059AF00B460028014E570240BF8E6B46102804302
:1059BF00E570240BF8E6B46211A870E8C0E0120994
:1059CF008BE4FBFA7980783F8018E570240BF8E6BA
:1059DF00B46317A870E8C0E012098BE4FBFA7920D2
:1059EF00784112019ED0E0F88034E570240BF8E680
:1059FF00B4682EE4FBFA79207840E8C0E0A8701272
:105A0F00098BD0E0F81202A7E4FBFA79A0784112D3
:105A1F00019EE4FBFA792078C11200ADA87012093B
:105A2F00FCE570240BF8E6FF64616009EF646360C6
:105A3F0004EFB4682A7F007E507DC37C47A87012A4
:105A4F0009A312019EE4FBFAF9783F1200AD12038D
:105A5F00EFEC1203B17B007A5079C3784780287F2F
:105A6F00007E247D747C49A8701209A312019EE464
:105A7F00FBFAF9783F1200AD1203EFEC1203B17B82
:105A8F00007A24797478491202A7A8701209FCA829
:105A9F007012098BE5702410F8CBE6CB08E6FA08F4
:0B5AAF00E6F91209717F0480027F00FD
:075ABA00E5702413F57022D2
:1049E1001570A870EBF61570A870EDF61570A8702B
:0849F100EFF6E57024F1F5700A
:1049F9002410F8E664016003024A8DE5702411F879
:0C4A0900E6FFE5702412127B31127F7D65
:104A1500E570240DF87664E570240DF8E6D394006E
:104A25004023E570240EF87603E570240EF8E6D3EE
:104A35009400400900E570240EF81680ECE570241A
:054A45000DF81680D2FF
:104A4A007D0F7F02127F88E5702412F8E6FFE57079
:104A5A002411F8E675F008A42FF582E435F0F58301
:104A6A00E5822400F582E5833400F583E4F0EF253E
:104A7A00E025E02490F582E43403F583120A2D3F01
:104A8A00800000E5702410F8E664026003024B50CF
:104A9A00E5702413F8E664086003024B50E57024BD
:104AAA0014F8CBE6CB08E6FA08E6F9120921E57014
:104ABA002412F8E6FB25E025E02490F582E434038D
:104ACA00F583120A08EB25E025E02490F582E43408
:104ADA0003F583E0FCA3E0FDA3E0FEA3E0FF7B0A6D
:104AEA007AD77923783C1203446002502AE570246D
:104AFA0012F8E625E025E02490F582E43403F583F4
:104B0A00E0FCA3E0FDA3E0FEA3E0FFE4FBFA7920CA
:104B1A007841120344502FE5702412F8E625E02567
:104B2A00E02490F582E43403F583120A2D3F8000D5
:104B3A0000E5702414F8CBE6CB08E6FA08E6F91289
:104B4A000A5E3F800000E5702410F8E66403600303
:104B5A00024E8BE5702413F8E6D3940740057F00D4
:104B6A00024E8DE5702411F8E6FFE57024121297C3
:104B7A00ADE5702408F8E65401D3940040057F009F
:104B8A00024E8DE5702412F8E6FDE5702411F8E670
:104B9A00FE75F008A42DF582E435F0F583E582244C
:104BAA0000F582E5833400F583E0FFE5702413F80D
:104BBA00E66F60057F00024E8DCFEECF127B341276
:104BCA00764BE5702412F8E6FFE5702411F8E6FE4C
:104BDA0075F008A42FF582E435F0F583E582240008
:104BEA00F582E5833400F583E0045407FD75F00887
:104BFA00EEA42FF582E435F0F583E5822400F582F0
:104C0A00E5833400F583EDF0E5702412F8E6FFE55C
:104C1A00702411F8E675F008A42FF582E435F0F552
:104C2A0083E5822400F582E5833400F583E0C454E9
:104C3A00F0440FFD7F02127F88E5702409F81209FB
:104C4A008BE41203B1E4FBFA7980784B1202A77B5A
:104C5A000A7AD77923784012019EA8701209FCA813
:104C6A007012098BE5702404F81209FCE57024130C
:104C7A00F8E6D39400403BA870E8C0E012098BE53F
:104C8A00702411F8E675F008A4FBE5702412F8EB1D
:104C9A002625E025E024F0F582E43403F583E0F8E4
:104CAA00A3E0F9A3E0FAA3E0FB1200A9D0E0F8120E
:104CBA0009FCE5702404F812098BE5702411F8E662
:104CCA0075F008A4FBE5702412F8EB2625E025E030
:104CDA0024F0F582E43403F583120A08A870E8C0C8
:104CEA00E012098BECC0E0EDC0E0EEC0E0EFC0E0FE
:104CFA00E5702412F8E625E025E02490F582E434F4
:104D0A0003F583E0FCA3E0FDA3E0FEA3E0FF7B6FD5
:104D1A007A127983783A12019EC8ECC8C9EDC9CAD9
:104D2A00EECACBEFCBD0E0FFD0E0FED0E0FDD0E082
:104D3A00FC1202A7D0E0F81209FCE570240FF8E68D
:104D4A00B47318A870E8C0E012098BE4FBFA792062
:104D5A0078411202A7D0E0F81209FC7F757E787DAF
:104D6A000C7C35A8701209A312019EA8701209A31F
:104D7A0012019EA8701209A312019EECC0E0EDC0B8
:104D8A00E0EEC0E0EFC0E07FFA7EED7D6B7C3AA8F2
:104D9A00701209A312019EA8701209A312019ED0D3
:104DAA00E0FBD0E0FAD0E0F9D0E0F81200ADECC0B8
:104DBA00E0EDC0E0EEC0E0EFC0E07F177ED97D16DF
:104DCA007C40A8701209A312019ED0E0FBD0E0FA41
:104DDA00D0E0F9D0E0F81200AD7BD37A4D79E278D1
:104DEA00411200ADA8701209FCA870E8C0E01209CF
:104DFA008B7B337A93798878431200A9D0E0F81232
:104E0A0009FCE4FFFE7D207C41A8701209A312016F
:104E1A009EE4FBFAF9783F1200AD1203EFEC12039D
:104E2A00B1E4FBFA792078411202A7A8701209FCB2
:104E3A007F007EC07D797C44A8701209A3120344C6
:104E4A00600B4009A870120A144479F99AE4FFFE2B
:104E5A007D487CC3A8701209A31203445009A870A4
:104E6A00120A14C479F99AA87012098BE5702414ED
:104E7A00F8CBE6CB08E6FA08E6F91209717F048056
:034E8A00027F01A3
:074E8D00E5702417F5702207
:1044C9001570A870EBF61570A870EDF61570A87048
:0844D900EFF6E57024F4F57024
:1044E100240DF8E66401600302456DE570240EF8C1
:0C44F100E6FFE570240F127B31127F7D86
:1044FD00E570240AF87664E570240AF8E6D3940092
:10450D004023E570240BF87603E570240BF8E6D311
:10451D009400400900E570240BF81680ECE570243A
:05452D000AF81680D21F
:10453200E570240CF8E6B477047D8880027D8C7FD8
:1045420002127F88E570240FF8E6FFE570240EF86A
:10455200E675F008A42FF582E435F0F583E58224B0
:1045620000F582E5833400F583E4F0E570240DF86C
:10457200E6640360030249D8E5702410F8E6D39498
:104582000240057F000249DAE570240EF8E6FFE5F5
:1045920070240FF8E6FD7B00E5702404F97A00121E
:1045A20097B9E5702404F8E65401D3940040057FDE
:1045B200000249DAE570240FF8E6FDE570240EF8F2
:1045C200E6FE75F008A42DF582E435F0F583E58268
:1045D2002400F582E5833400F583E0FFE5702405CD
:1045E200F8EFF65401FFE5702410F8EF6660057FDE
:1045F200000249DACFEECF127B347B00E57024064D
:10460200127651E570240CF8E6647760030246A73F
:10461200E570240FF8E6FFE570240EF8E6FE75F06B
:1046220008A42FF582E435F0F583E5822400F582B3
:10463200E5833400F583E0045401FD75F008EEA42F
:104642002FF582E435F0F583E5822400F582E583D7
:104652003400F583EDF0E570240FF8E6FF75F008FD
:10466200EEA42FF582E435F0F583E5822400F5828D
:10467200E5833400F583E070047D8880027D987FB5
:1046820002127F88E5702406F812098BE41203B146
:10469200E4FBFA7980784B1202A77B0A7AD779A3D6
:1046A200783C024737E570240FF8E6FFE570240EE8
:1046B200F8E6FE75F008A42FF582E435F0F583E5FF
:1046C200822400F582E5833400F583E0045401FD81
:1046D20075F008EEA42FF582E435F0F583E5822427
:1046E20000F582E5833400F583EDF0E570240FF8E0
:1046F200E6FF75F008EEA42FF582E435F0F583E5C8
:10470200822400F582E5833400F583E0C454F0444A
:104712008CFD7F02127F88E5702406F812098BE473
:104722001203B1E4FBFA7980784B1202A77B0A7A72
:10473200D779A3783E12019EA8701209FCE5702475
:104742000CF8E6FF64756008EF6476600302483394
:10475200A870E8C0E012098B7B6F7A127983783AED
:104762001202A7D0E0F81209FCE570240CF8E6B4B6
:104772007618A870E8C0E012098BE4FBFA79207879
:10478200411202A7D0E0F81209FC7F757E787D0CF9
:104792007C35A8701209A312019EA8701209A312F7
:1047A200019EA8701209A312019EECC0E0EDC0E0C8
:1047B200EEC0E0EFC0E07FFA7EED7D6B7C3AA87040
:1047C2001209A312019EA8701209A312019ED0E041
:1047D200FBD0E0FAD0E0F9D0E0F81200ADECC0E096
:1047E200EDC0E0EEC0E0EFC0E07F177ED97D167C21
:1047F20040A8701209A312019ED0E0FBD0E0FAD0CB
:10480200E0F9D0E0F81200AD7BD37A4D79E278413D
:104812001200ADA8701209FCA870E8C0E012098B62
:104822007B337A93798878431200A9D0E0F8024961
:1048320056E570240CF8E664776003024959A870C3
:10484200E8C0E012098B7B007A247974784912015E
:104852009ED0E0F81209FC7F5D7E0B7D237C2CA8A4
:10486200701209A312019EA8701209A312019EA838
:10487200701209A312019EA8701209A312019EECE4
:10488200C0E0EDC0E0EEC0E0EFC0E07F177EEE7D5D
:104892008B7C32A8701209A312019EA8701209A380
:1048A20012019EA8701209A312019EC8ECC8C9ED9C
:1048B200C9CAEECACBEFCBD0E0FFD0E0FED0E0FD1C
:1048C200D0E0FC1200A9ECC0E0EDC0E0EEC0E0EFE9
:1048D200C0E07F4B7E5F7D047C38A8701209A31272
:1048E200019EA8701209A312019ED0E0FBD0E0FA4B
:1048F200D0E0F9D0E0F81200ADECC0E0EDC0E0EE9F
:10490200C0E0EFC0E07F4B7E767D6C7C3DA87012EC
:1049120009A312019ED0E0FBD0E0FAD0E0F9D0E08A
:10492200F81200AD7B1F7A85796B78BE1200ADA8B4
:10493200701209FCE4FFFEFDFCA8701209A3120329
:10494200446014A8701209A3E4FFFE7D7A7C44122D
:1049520002A7A8701209FCE4FFFE7DC87C42A87081
:104962001209A312019EE4FBFAF9783F1200AD127C
:1049720003EFEC1203B1E4FBFA79C878421202A702
:10498200A8701209FC7F5C7EFF7D797C44A87012BE
:1049920009A3120344600B4009A870120A14447957
:1049A200FF5CE4FFFE7D207CC1A8701209A3120304
:1049B200445009A870120A14C11FD70AA87012091C
:1049C2008BE5702411F8CBE6CB08E6FA08E6F9127B
:0849D20009717F0480027F01DE
:0749DA00E5702414F57022C2
:10677C001570A870EBF61570A870EDF61570A87072
:08678C00EFF6E57024F5F5704D
:10679400E570240CF8E66401600302682AE57024BD
:0E67A4000DF8E6FFE570240E127B31127F7DAA
:1067B200E5702409F87664E5702409F8E6D39400BC
:1067C2004023E570240AF87603E570240AF8E6D33C
:1067D2009400400900E570240AF81680ECE5702464
:0567E20009F81680D249
:1067E7007D057F02127F88E570240EF8E6FFE570CD
:1067F700240DF8E675F008A42FF582E435F0F5834B
:10680700E5822400F582E5833400F583E4F0EF2583
:10681700E025E02490F582E43403F583120A2D3F46
:10682700800000E570240CF8E664036003026A3414
:10683700E570240FF8E6D3940740057F00026A3617
:10684700E570240DF8E6FFE570240EF8E6FD7B0001
:10685700E5702404F97A001297B9E5702404F8E684
:106867005401D3940040057F00026A36E570240E78
:10687700F8E6FDE570240DF8E6FE75F008A42DF5A1
:1068870082E435F0F583E5822400F582E583340060
:10689700F583E0FFE570240FF8E66F60057F0002DF
:1068A7006A36CFEECF127B347B00E5702405127673
:1068B70051E570240EF8E6FFE570240DF8E6FE7545
:1068C700F008A42FF582E435F0F583E5822400F57E
:1068D70082E5833400F583E0045407FD75F008EE84
:1068E700A42FF582E435F0F583E5822400F582E5EF
:1068F700833400F583EDF0E570240EF8E6FFE570CC
:10690700240DF8E675F008A42FF582E435F0F58339
:10691700E5822400F582E5833400F583E0C454F072
:106927004405FD7F02127F88E5702405F812098B64
:10693700E41203B1E4FBFA7980784B1202A77B0AD1
:106947007AD779A3783F12019EC8ECC8C9EDC9CAA6
:10695700EECACBEFCB7F0A7ED77D237C3F1200A9FF
:10696700A8701209FCA870E8C0E012098BE4FBFAD2
:10697700797A78441202A7D0E0F81209FCA870E8E7
:10698700C0E012098B7B007A247974784912019E42
:10699700D0E0F81209FCA870E8C0E012098B7B9AD6
:1069A7007A99798878431200A9D0E0F81209FCE4B3
:1069B700FFFE7DC87C42A8701209A312019EE4FB6A
:1069C700FAF9783F1200AD1203EFEC1203B1E4FBC2
:1069D700FA79C878421202A7A8701209FCE4FFFEF0
:1069E7007D167C43A8701209A3120344600B40096B
:1069F700A870120A144479FF5CE4FFFE7D5C7CC238
:106A0700A8701209A31203445009A870120A14C4EB
:106A170079FF5CA87012098BE5702410F8CBE6CBE0
:0F6A270008E6FA08E6F91209717F0480027F0180
:076A3600E5702413F5702246
:0C98E5007F011280DD7FFC1298F17F00F3
:0898F1001570A870EFF6157068
:1098F900C2B3C2B100000000000000000000000077
:109909000000000000000000A870E4F6A870E6C39B
:1099190094085047D2B008E6FF548094004003D31E
:109929008001C392B30000000000000000000000A5
:10993900000000000000000000C2B00000000000AC
:10994900000000000000000000000000000000A866
:109959007008EF25E0F6A8700680B1D2B1C2B30055
:1099690000000000000000000000000000000000EE
:03997900000000EB
:05997C000570057022DA
:1080DD001570A870EDF61570A870EFF61570157087
:1080ED00C2B3C2B10000000000000000000000009B
:1080FD000000000000000000A8700808E62450A849
:10810D007008F6A870E4F6A870E6C394085047D23C
:10811D00B008E6FF548094004003D38001C392B3AE
:10812D000000000000000000000000000000000042
:10813D0000000000C2B000000000000000000000C0
:10814D0000000000000000000000A87008EF25E00E
:10815D00F6A8700680B1A8700808E62450A870082B
:10816D00F6A870E4F6A870E6C394085040D2B0C2E9
:10817D00B30000000000000000000000000000003F
:10818D000000000000C2B000000000000000000070
:10819D00000000000000000000000008E8C0E0E65C
:1081AD0025E0FFD0E0F8EFF6A8700680B8A870E4DF
:1081BD00F6A870E6C39408504ED2B0E5702403F8CB
:1081CD00E6FF5480D394004003D38001C392B300E3
:1081DD000000000000000000000000000000000092
:1081ED00000000C2B0000000000000000000000010
:1081FD00000000000000000000E5702403F8EF25EA
:10820D00E0F6A8700680AAD2B1C2B300000000004B
:0F821D0000000000000000000000000000000052
:07822C00E5702404F5702247
:107E1700157015701570A870C6EBC608C6EAC608B7
:097E2700C6E9C6E57024FCF57003
:107E3000C2B10000000000000000000000000000CF
:107E4000000000000000F8087601A870E4F6A870B1
:107E5000E6C394085047D2B008E6FF54809400402F
:107E600003D38001C392B3000000000000000000B3
:107E70000000000000000000000000C2B000000090
:107E800000000000000000000000000000000000F2
:0D7E900000A87008EF25E0F6A8700680B18C
:107E9D00A87008087605A8700808E6D3940040225B
:107EAD00E5702403F87613E5702403F8E6D3940007
:107EBD00400900E5702403F81680ECA87008081638
:027ECD0080D45F
:107ECF00A870E4F6E5702404F8CBE6CB08E6FA08D0
:107EDF00E6F9120A5E00000000A870E6C39418507D
:107EEF0070D2B00000000000000000000000000091
:107EFF0000000000000000E5702404F8CBE6CB087A
:107F0F00E6FA08E6F9120921780112090EC8ECC841
:107F1F00C9EDC9CAEECACBEFCBA2B4E4334BFFEA2B
:107F2F00FEE9FDE8FCE5702404F8CBE6CB08E6FAA1
:107F3F0008E6F9120971C2B000000000000000004D
:107F4F00000000000000000000000000A870068084
:107F5F0088D2B10000000000000000000000000007
:077F6F00000000000000000B
:077F7600E5702407F57022FD
:105AC1001570A870EBF61570A870EDF61570A8703A
:085AD100EFF6E57024F6F57014
:105AD900240BF8E664016003025BB0E570240CF85E
:105AE900E6FFE570240D12AC627D027F001280DDB5
:105AF9001D7F021280DD7DD07F031280DD7FF012D1
:105B090098F1E5702404F8120A14000000007FA03F
:105B19007E867D017C00E5702404F81209A3C31276
:075B290008FD505730B55490
:105B3000E5702408F87601E5702408F8E6D39400AF
:105B40004023E5702409F87603E5702409F8E6D3CC
:105B50009400400900E5702409F81680ECE57024F3
:055B600008F81680D2D8
:105B6500E5702404F812098BEF2401FFE43EFEE4FE
:105B75003DFDE43CFCE5702404F81209FC80937DAE
:105B85000F1298E5E570240DF8E6FFE570240CF892
:105B9500E675F008A42FF582E435F0F583E5822457
:105BA50040F582E5833405F583E4F0E570240BF8D0
:105BB500E664036003025E3DE570240EF8E6D394C7
:105BC5000740057F00025E3FE570240CF8E6FFE51F
:105BD50070240D12AC62E5702404F8120A1400005A
:105BE5000000E47F107E27FDFCE5702404F812090F
:0A5BF500A3C31208FD505730B55449
:105BFF00E5702408F87601E5702408F8E6D39400E0
:105C0F004023E5702409F87603E5702409F8E6D3FC
:105C1F009400400900E5702409F81680ECE5702423
:055C2F0008F81680D208
:105C3400E5702404F812098BEF2401FFE43EFEE42E
:105C44003DFDE43CFCE5702404F81209FC8094E476
:105C54007F107E27FDFCE5702404F81209A3C3120B
:105C640008FD7004FF025E3FE570240DF8E6FEE5D2
:105C740070240CF8E675F008A42EF582E435F0F5EE
:105C840083E5822440F582E5833405F583E0FDE570
:105C940070240EF8E66D60057F00025E3FE5702417
:105CA4000DF8E6FFE570240CF8E6FCED045407FD5E
:105CB40075F008ECA42FF582E435F0F583E5822431
:105CC40040F582E5833405F583EDF075F008ECA426
:105CD4002EF582E435F0F583E5822440F582E583F0
:105CE4003405F583E0C454F0440FFD1298E57B00BD
:105CF400E5702404F97A00127E17E5702404F81282
:105D0400098B780812090EEC1203B1A8701209FC71
:105D1400E4FBFA7980784FE8C0E0A87012098BD0D0
:105D2400E0F81202A7E4FBFA79A0784012019EA8D9
:105D3400701209FCE570240AF8E6B46402803FE5B9
:105D440070240AF8E6B4652DE4FBFA79207840E87B
:105D5400C0E0A87012098BD0E0F81202A7E4FBFAA5
:105D640079A0784112019EE4FBFA792078C11200EF
:105D7400ADA870803EE570240AF8E6B46617A870F2
:105D8400E8C0E012098BE4FBFA7980783F12019EA7
:105D9400D0E0F8801EE570240AF8E6B46718A8700D
:105DA400E8C0E012098BE4FBFA7920784112019EE5
:105DB400D0E0F81209FCE570240AF8E6FF64656097
:105DC40004EFB4672A7F007E407D1C7C46A87012D5
:105DD40009A312019EE4FBFAF9783F1200AD120305
:105DE400EFEC1203B17B007A40791C784680287F5F
:105DF400007E507DC37C47A8701209A312019EE463
:105E0400FBFAF9783F1200AD1203EFEC1203B17BF9
:105E1400007A5079C378471202A7A8701209FCA827
:105E24007012098BE570240FF8CBE6CB08E6FA086C
:0B5E3400E6F91209717F0480027F0173
:075E3F00E5702412F570224A
:106CF0001570A870EBF61570A870EDF61570A870F9
:086D0000EFF6E57024F5F570D3
:106D0800240CF8E664036003026F93E570240FF81F
:106D1800E6FED3940340057F00026F957401C8EE28
:106D2800C8088002C333D8FCA8700808F675840127
:106D3800E5702403F8120A1400000000A870E4F6B5
:106D4800A870E6C3940A4003026E00E4F5CCF5CDC2
:106D5800F5C975C804E570240DF8E6FFE570240E42
:106D680012AC62E570240DF8E6FFE570240EF8E633
:106D7800FDE4FB12AC677F0012AA28E570240DF829
:106D8800E6FFE570240EF8E6FD7B00A970097A009D
:106D98001297B9A8700808C9E8C9A87008E657602A
:106DA80005E5C830E7D0E4F5C8E5702403F8E8C085
:106DB800E012098BECC0E0EDC0E0EEC0E0EFC0E00F
:106DC800AFCDEFFEADCC7C00E42DFFEC3ECBEFCB9E
:106DD800FAE4F9F8D0E0FFD0E0FED0E0FDD0E0FC26
:106DE800EF2BFFEE3AFEE93DFDE83CFCD0E0F8125F
:106DF80009FCA87006026D48E5C85480FFBF01274A
:106E0800E570240BF8E6B4700FE5702407F8120A51
:106E180014411FFFFF026F76E5702407F8120A1469
:106E28004479FFFE026F76E5702403F812098BE4BB
:106E38001203B1ECC0E0EDC0E0EEC0E0EFC0E0A8A6
:106E480070E6FCE41203BBC8ECC8C9EDC9CAEECAB7
:106E5800CBEFCBD0E0FFD0E0FED0E0FDD0E0FC12DD
:106E680002A7E4FBFA79C478421202A7E4FBFA7994
:106E780040784112019EE5702407F81209FCE5707C
:106E88002407F8E8C0E012098B7B007A247974782B
:106E9800491202A7D0E0F81209FCE570240BF8E6C5
:106EA80064707BCD7ACC798C783F7044E8C0E0E59B
:106EB800702407F812098BD0E0F81202A77B007A39
:106EC800B8790878491202A77B287A6B796E784ED0
:106ED80012019EE5702407F81209FCE5702407F8F2
:106EE800E8C0E012098B7B777ABE799F783D8041B4
:106EF800E8C0E0E5702407F812098BD0E0F8120228
:106F0800A7E4FBFA79AF78451202A77B287A6B7958
:106F18006E784E12019EE5702407F81209FCE570A0
:106F28002407F8E8C0E012098B7B9A7A9979F978F6
:106F3800401200A9D0E0F81209FCE4FFFE7D7A7C3B
:106F480044E5702407F81209A312019EE4FBFAF93C
:106F5800783F1200AD1203EFEC1203B1E4FBFA79AB
:106F68007A78441202A7E5702407F81209FCE57044
:106F78002407F812098BE5702410F8CBE6CB08E655
:0D6F8800FA08E6F91209717F0480027F010A
:076F9500E5702413F57022E2
:10166F001570A870EBF61570A870EDF61570A870D0
:08167F00EFF6E57024F0F570B0
:10168700E5702412F8E675F008A4FFE5702413F856
:10169700EF26FFE570240DF8EFF6E5702411F8E664
:1016A700640460030217C7E5702414F8E67032E596
:1016B70070240DF8E625E025E02450F582E4340493
:1016C700F583120A2D42960000E5702415F8CBE643
:1016D700CB08E6FA08E6F9120A5E429600000217FE
:1016E700C2E5702414F8E6B40132E570240DF8E67B
:1016F70025E025E024E8F582E43405F583120A2D78
:1017070000000000E5702415F8CBE6CB08E6FA08E0
:10171700E6F9120A5E000000000217C2E570241401
:10172700F8E6B40231E570240DF8E625E025E0245B
:10173700B0F582E43404F583120A2D3F800000E5FA
:10174700702415F8CBE6CB08E6FA08E6F9120A5E2C
:101757003F8000008065E5702414F8E6FFB4032B92
:10176700E570240DF8E625E02410F582E43405F54C
:1017770083E4F0A3743CF0E5702415F8CBE6CB08BE
:10178700E6FA08E6F9E475F03C802DEFB4042CE5A1
:1017970070240DF8E625E02460F582E43409F5832A
:1017A700E4F0A37405F0E5702415F8CBE6CB08E662
:1017B700FA08E6F9E475F0051208BA7F00021FD8A7
:1017C700E570240DF8E62490F582E43409F583E00A
:1017D700600302189E12ACBDE570240DF8E625E003
:1017E70025E02458F582E43405F583E0F8A3E0F911
:1017F700A3E0FAA3E0FBC3EF9BFFEE9AFEED99FD92
:10180700EC98FCECC0E0EDC0E0EEC0E0EFC0E0E536
:1018170070240DF8E625E02410F582E43405F583FD
:10182700E0FEA3E0FF7C007D64120782CBEFCBCA0A
:10183700EECAE4F9F8D0E0FFD0E0FED0E0FDD0E05A
:10184700FCC31208FD400302197AE570240DF8E67F
:101857002490F582E43409F5837401F012ACBDE5F8
:1018670070240DF8E6FB25E025E02458F582E434E2
:1018770005F583120A08EB25E025E02450F582E4FC
:101887003404F583E0FCA3E0FDA3E0FEA3E0FFA89A
:10189700701209FC02194312ACBDE570240DF8E67D
:1018A70025E025E02458F582E43405F583E0F8A324
:1018B700E0F9A3E0FAA3E0FBC3EF9BFFEE9AFEED8E
:1018C70099FDEC98FCECC0E0EDC0E0EEC0E0EFC0A5
:1018D700E0E570240DF8E625E02460F582E434099C
:1018E700F583E0FEA3E0FF7C007D64120782CBEF67
:1018F700CBCAEECAE4F9F8D0E0FFD0E0FED0E0FDB5
:10190700D0E0FCC31208FD506AE570240DF8E62408
:1019170090F582E43409F583E4F012ACBDE5702458
:101927000DF8E625E025E02458F582E43405F58333
:10193700120A08A870120A1400000000A970157096
:1019470015701570A870760008760008C6E9C615E8
:1019570070A870E4F6E5702417F8E61570A870F61D
:10196700E5702417F8E6FB7D02E5702415F8E6FF1D
:1019770012166FE5702411F8E664016003021A1A63
:10198700E5702412F8E6FFE5702413F8E6FD7B0EF8
:10199700129C66E5702412F8E6FFE5702413F8E65A
:0C19A700FD7B0E1295DE127B26127F7D68
:1019B300E570240EF87664E570240EF8E6D39400FF
:1019C3004023E570240FF87603E570240FF8E6D37F
:1019D3009400400900E570240FF81680ECE57024AC
:0519E3000EF81680D291
:1019E8007D077F02127F88E570240DF8E62490F5C4
:1019F80082E43409F5837401F012ACBDE570240D5E
:101A0800F8E625E025E02458F582E43405F583124C
:101A18000A08E5702411F8E664026003021CF0E588
:101A2800702414F8E6703FE5702415F8CBE6CB086F
:101A3800E6FA08E6F9120921E4FBFAF9F812034478
:101A48005024E5702415F8CBE6CB08E6FA08E6F949
:101A5800120921E570240DF8E625E025E02450F56B
:101A680082E434048058E5702414F8E6B40124E5CF
:101A7800702415F8CBE6CB08E6FA08E6F912092136
:101A8800E570240DF8E625E025E024E8F582E43445
:101A980005802BE5702414F8E6B40229E5702415B6
:101AA800F8CBE6CB08E6FA08E6F9120921E5702436
:101AB8000DF8E625E025E024B0F582E43404F5834A
:101AC800120A088062E5702414F8E6FFB4032BE5D7
:101AD800702415F8CBE6CB08E6FA08E6F912081FD9
:101AE800FDE570240DF8E625E02410F582E43405C0
:101AF800F583E5F0F0A3EDF0802DEFB40429E5704F
:101B08002415F8CBE6CB08E6FA08E6F912081FFF19
:101B1800E570240DF8E625E02460F582E43409F543
:101B280083E5F0F0A3EFF0E5702414F8E6D3940011
:101B380040057F00021FD8E5702415F8CBE6CB08D6
:101B4800E6FA08E6F9120921A8701209FCE4FFFE7A
:101B5800FDFCA8701209A31203445009A870120AC8
:101B68001400000000E4FFFE7DC87C42A870120942
:101B7800A3120344600B4009A870120A1442C8005B
:101B880000E4FBFA79C87842E8C0E0A87012098B33
:101B9800D0E0F81202A77B007AFF797F784712011C
:101BA8009E1203EFE570240AF8EEF608EFF6E570EA
:101BB8002412F8E6FFE5702413F8E6FDE4FB12951D
:101BC800DEE570240CF8E4F6E570240CF8E6FFC3B3
:101BD80094045033EF940140047F0480027F001284
:101BE80095C2E5702412F8E6FFE5702413F8E6FDC7
:101BF800E5702405F8E64408FB1295DE1295C9E560
:101C080070240CF80680C1E570240CF8E4F6E57041
:101C1800240CF8E6C39404504DE5702414F8E654F7
:101C280008D3940040047F0480027F001295C2E527
:101C3800702412F8E6FFE5702413F8E6FDE5702439
:101C480005F8E64408FB1295DE1295C9E5702414E0
:101C5800F8E8C0E0E625E0FFD0E0F8EFF6E570240C
:101C68000CF806021C16E570240CF8E4F6E570245E
:101C78000CF8E6C39410505DE570240AF8E6548029
:101C8800FED3E49400EE940040047F0480027F00B9
:101C98001295C2E5702412F8E6FFE5702413F8E601
:101CA800FDE5702405F8E64408FB1295DE1295C997
:101CB800E570240AF8E8C0E0C9E8C909E725E0FFAB
:101CC80019E733FED0E0F8EEF608EFF6E570240CDD
:101CD800F806021C75E5702412F8E6FFE570241377
:101CE800F8E6FD7B0E1295DEE5702411F8E6640334
:101CF8006003021FD6E5702414F8E67013E570241B
:101D08000DF8E625E025E02450F582E43404803619
:101D1800E5702414F8E6B40113E570240DF8E625FF
:101D2800E025E024E8F582E43405801AE5702414FF
:101D3800F8E6B40221E570240DF8E625E025E02454
:101D4800B0F582E43404F583E0FCA3E0FDA3E0FEF3
:101D5800A3E0FF021FBDE5702414F8E6FEB40328D3
:101D6800E570240DF8E625E02410F582E43405F545
:101D780083E0F9A3E0FDE5702415F8CBE6CB08E68F
:101D8800FA08E6C98DF0802AEEB4042EE570240D19
:101D9800F8E625E02460F582E43409F583E0F9A348
:101DA800E0FFE5702415F8CBE6CB08E6FA08E6C9AB
:101DB8008FF01208BA7F02021FD8E5702414F8E6E3
:101DC800640560057F00021FD8E5702412F8E6FF5D
:101DD800E5702413F8E6FD7B00E5702404F97A0029
:101DE8001297B9E5702404F8E65401D3940040052D
:101DF8007F00021FD8127B267B00E570240612762E
:101E0800517D077F02127F88E5702406F812098B3E
:101E1800E41203B1E4FBFA7980784B1202A77B0A3B
:101E28007AD779A3784012019E7B0A7AD7792378EA
:101E3800C01200ADA8701209FCA870E8C0E0120931
:101E48008B7B387A1F7943784112019ED0E0F812D3
:101E580009FCA870E8C0E012098BECC0E0EDC0E016
:101E6800EEC0E0EFC0E0E570240DF8E625E025E0DF
:101E78002450F582E43404F583E0FCA3E0FDA3E0FC
:101E8800FEA3E0FFE4FBFA797A78441202A7C8ECD3
:101E9800C8C9EDC9CAEECACBEFCBD0E0FFD0E0FE8F
:101EA800D0E0FDD0E0FC1202A7D0E0F81209FC7BDC
:101EB800CD7ACC792C7840E8C0E0A87012098BD094
:101EC800E0F81202A7C8ECC8C9EDC9CAEECACBEF40
:101ED800CBE4FFFE7DC87C421200A9A8701209FC61
:101EE800E570240DF8E625E025E024E8F582E434E1
:101EF80005F583E0F8A3E0F9A3E0FAA3E0FBE8C066
:101F0800E0A87012098BD0E0F81200A9E570240D42
:101F1800F8E625E025E024B0F582E43404F583E012
:101F2800F8A3E0F9A3E0FAA3E0FB12019EA870125F
:101F380009FC7F007E507DC37C47A8701209A3125C
:101F4800019EE4FBFAF9783F1200AD1203EFEC12A0
:101F580003B17B007A5079C378471202A7A87012A0
:101F680009FCE570240DF8E62490F582E43409F5BF
:101F780083E06401705412ACBDE570240DF8E625C9
:101F8800E025E02458F582E43405F583E0F8A3E081
:101F9800F9A3E0FAA3E0FBC3EF9BFFEE9AFEED99ED
:101FA800FDEC98FCE47B64FAF9F8C31208FD501ABA
:101FB800A87012098BE5702415F8CBE6CB08E6FA71
:101FC80008E6F91209717F0480067F0080027F010C
:071FD800E5702418F57022EA
:106F9C001570A870EBF61570A870EDF61570A8704A
:086FAC00EFF6E57024F5F57025
:106FB400E570240CF8E664017021E570240DF8E610
:106FC400FFE570240EF8E6FD7BFF1295DEE57024E4
:106FD4000DF8E6FFE570240E129C61E570240CF8B0
:106FE400E664036003027235E570240FF8E670125C
:106FF400E570240DF8E6FFE570240EF8E6FD7BFE4F
:107004008010E570240DF8E6FFE570240EF8E6FD27
:107014007BFD1295DEE570240DF8E6FFE570240E85
:0370240012AC6249
:10702700E5702409F8760AE5702409F8E6D3940098
:107037004023E570240AF87603E570240AF8E6D3BE
:107047009400400900E570240AF81680ECE57024E6
:0570570009F81680D2CB
:10705C0030B418E570240DF8E6FFE570240EF8E660
:10706C00FD7BFF1295DE7F00027237E5702404F879
:10707C00120A1400000000E5702408F8E4F6E5702C
:10708C002408F8E6C3941B507500000000000000B3
:10709C0000000000000000000000000000D2B00062
:1070AC0000000000000000000000000000000000D4
:1070BC00000000C2B0000000000000000000000052
:1070CC00000000000000000000E5702404F8120924
:1070DC008B780112090EC8ECC8C9EDC9CAEECACB2F
:1070EC00EFCBA2B4E4334BFFEAFEE9FDE8FCE5701C
:1070FC002404F81209FCE5702408F8068080E57079
:10710C00240DF8E6FFE570240EF8E6FD7BFF1295E2
:10711C00DEE5702404F812098BE4FFFEFDEC54024A
:10712C00FC601EE5702404F812098BE4FFFEFDECF4
:10713C005401FC600CA870120A144020000002716B
:10714C00D2E5702404F812098BE4FFFEFDEC540226
:10715C00FCE4FBFAF9F8C31208FD701DE570240479
:10716C00F812098BE4FFFEFDEC5401FC600BA870D7
:10717C00120A1400000000804DE5702404F8120976
:10718C008BE4FFFEFDEC5402FCE4FBFAF9F8C312AD
:10719C0008FD700CE5702404F812098B74FF80094B
:1071AC00E5702404F812098BE4FC1203B1E4FBFA39
:1071BC007980784B1202A7E4FBFA7920784012010F
:1071CC009EA8701209FCE4FFFEFD7C41A870120918
:1071DC00A312019EE4FBFA792078C11200ADA870CD
:1071EC001209FC7F007E247D747C49A8701209A3CF
:1071FC0012019EE4FBFAF9783F1200AD1295127B56
:10720C00007A24797478491202A7A8701209FCA894
:10721C007012098BE5702410F8CBE6CB08E6FA085F
:0B722C00E6F91209717F0480027F0068
:07723700E5702413F570223D
:0677F2008F448D458B461B
:1077F800E4FFFEFDFCAB4AAA49A948A84712034486
:107808005009E4F54AF549F548F547E4FFFE7D34AB
:107818007C43AB4AAA49A948A847120344600D40D3
:107828000BE4F54AF549754834754743AF4AAE4904
:10783800AD48AC47ECC0E0EDC0E0EEC0E0EFC0E022
:10784800E54575F008A47C002546FFEC35F0FEEF11
:107858007802C333CE33CED8F92460F58274063E5D
:10786800F583D0E0FFD0E0FED0E0FDD0E0FC120AC6
:1078780008E4FBFA79907842AF4AAE49AD48AC4784
:107888001202A7E4FBFA792078401202A77B007A5B
:10789800FF797F784712019E1203EF8E4B8F4C7B46
:1078A80048AD45AF441295DE7B06AD45AF4412ACFA
:1078B80067E4FDEDD394014003D38001C392B30084
:1078C80000000000000000000000000000000000B0
:1078D800000000D2B000000000000000000000001E
:1078E800000000000000000000C2B00DBD04C4E4A8
:1078F800FDE5465408D394004003D38001C392B3F6
:10790800000000000000000000000000000000006F
:1079180000000000D2B000000000000000000000DD
:1079280000000000000000000000C2B0E54625E0AD
:10793800F5460DBD04BBE4FDE54B5480FED3E4944D
:1079480000EE94004003D38001C392B3000000000E
:10795800000000000000000000000000000000001F
:10796800D2B000000000000000000000000000008D
:10797800000000000000C2B0E54C25E0F54CE54BE6
:1079880033F54B0DBD10B17B40AD45AF440295DEDC
:103127001570A870EBF61570A870EDF61570A870FD
:08313700EFF6E57024F0F570DD
:10313F00E5702412F8E6FF75F008A4FEE57024137D
:10314F00F8E6FD2EFEE570240DF8EEF6E57024117D
:10315F00F8E6640160030232457B78129C66E570E5
:10316F002412F8E6FFE5702413F8E6FD7B40129574
:10317F00DEE5702412F8E6FFE5702413F8E6FD7B18
:10318F00701295DEE5702412F8E6FFE57024131235
:0C319F00AC62127F7D7D117F07127F88DB
:1031AB00E570240EF87664E570240EF8E6D39400EF
:1031BB004023E570240FF87603E570240FF8E6D36F
:1031CB009400400900E570240FF81680ECE570249C
:0531DB000EF81680D281
:1031E0007D577F02127F88E5702413F8E6FEE570B4
:1031F0002412F8E6FF75F008A42EF582E435F0F508
:1032000083E58224B8F582E5833405F583E4F0751F
:10321000F008EFA42EF582E435F0F583E58224D0A2
:10322000F582E5833405F583E4F0E5702413F8E6D0
:10323000FD7B401295DE7E037F007D007B017A00DE
:103240007930120ADEE5702411F8E66402600302A8
:1032500032E1E5702414F8E6FED3940740057F00C0
:103260000238A5EE7029E5702415F8CBE6CB08E608
:10327000FA08E6F9E5702413F8E675F003A42430A3
:10328000F582E43403F583EBF0A3EAF0A3E9F0E57B
:10329000702415F8CBE6CB08E6FA08E6F912092106
:1032A000A8701209FCE5702412F8E6FFEFC0E0E513
:1032B000702413F8E6FDEDC0E0E5702414F8E6FB99
:1032C000A87012098B8F4A8E498D488C47D0E0FD3B
:1032D000D0E0FF1277F212ACBD8F178E168D158CD1
:1032E00014E5702411F8E6640360030238A3E57066
:1032F0002414F8E6FFC394084006EFD39417400562
:103300007F000238A5E5702412F8E6FFE57024136B
:103310001297ADE5702408F8E630E00302367AE54E
:10332000702413F8E6FDE5702412F8E6FE75F00847
:10333000A42DF582E435F0F583E58224B8F582E525
:10334000833405F583E02408FBE433FAE5702414A4
:10335000F8E66B7001EA60057F000238A5CFEECF7A
:103360007B501295DE127B2612764BE5702413F803
:10337000E6FFE5702412F8E6FE75F008A42FF5824A
:10338000E435F0F583E58224B8F582E5833405F56C
:1033900083E0045407FD75F008EEA42FF582E435B0
:1033A000F0F583E58224B8F582E5833405F583EDF5
:1033B000F0E5702413F8E6FFE5702412F8E675F0E6
:1033C00008A42FF582E435F0F583E58224B8F58270
:1033D000E5833405F583E0903F5893C454F04407E7
:1033E000FD7F02127F88E5702412F8E6FFE5702465
:1033F00013F8E6FD7B401295DEE5702409F812090A
:103400008BE41203B1E4FBFA7980784B1202A77BBC
:103410000A7AD779A3784012019E7B0A7AD779235A
:1034200078C01200ADA8701209FCA870E8C0E012C4
:10343000098BE4FBFA79CA784212019ED0E0F812B7
:1034400009FCE5702413F8E675F008A4FFE5702484
:1034500014F8E67C002FFFEC35F0FEEF7802C33362
:10346000CE33CED8F92410F58274003EF583E0FC0B
:10347000A3E0FDA3E0FEA3E0FFE5702404F8120939
:10348000FCE4FFFE7D807CBFE5702404F81209A3F4
:103490001203446048A870E8C0E012098BECC0E059
:1034A000EDC0E0EEC0E0EFC0E07F0A7ED77D237C78
:1034B0003CE5702404F81209A312019EC8ECC8C9A7
:1034C000EDC9CAEECACBEFCBD0E0FFD0E0FED0E032
:1034D000FDD0E0FC1200A9D0E0F81209FCE4FFFEE8
:1034E0007D7A7C44A8701209A312019EE4FBFAF9CC
:1034F000783F1200AD1203EFEC1203B1E4FBFA794E
:103500007A78441202A7A8701209FCA87012098BDD
:10351000E5702415F8CBE6CB08E6FA08E6F91209BF
:103520007112ACBDC8ECC8C9EDC9CAEECACBEFCBAD
:10353000E5172432FFE43516FEE43515FDE43514B5
:10354000FCD31208FD5003023675E5702414F8E62A
:1035500024F8FFE434FFFEEF7802C333CE33CED835
:10356000F9FFE5702413F8E675F003A42430F58222
:10357000E43403F583E0FBA3E0FAA3E0F98F828E45
:10358000831209CCE8C0E0A87012098BD0E0F812D1
:1035900000A9E5702404F81209FCE5702404F8126F
:1035A000098B12AD227B6F7A127983783A12034429
:1035B0004003023675E5702404F812098B12AD221F
:1035C000E4FBFA79A078401203446002500302360B
:1035D00075E4FFFEFD7C40E5702404F81209A31297
:1035E0000344600E400CE5702404F8120A144000F5
:1035F0000000E4FFFEFD7CC0E5702404F81209A37E
:10360000120344500CE5702404F8120A14C00000A0
:1036100000E5702413F8E675F008A4FFE5702414A3
:10362000F8E67C002FFFEC35F0FEEF7802C333CED6
:1036300033CED8F92440F58274063EF583E0FCA32E
:10364000E0FDA3E0FEA3E0FFE5702404F81209A367
:103650001200A98F4A8E498D488C47E5702412F8D4
:10366000E6FFE5702413F8E6FDE5702414F8E6247F
:10367000F8FB1277F27F040238A5E5702408F8E61B
:1036800030E10302389FE5702413F8E6FDE570246D
:1036900012F8E6FE75F008A42DF582E435F0F58306
:1036A000E58224D0F582E5833405F583E02410FB20
:1036B000E433FAE5702414F8E66B7001EA60057FE4
:1036C000000238A5CFEECF7B601295DE127B26126A
:1036D000764BE5702413F8E6FFE5702412F8E6FE59
:1036E00075F008A42FF582E435F0F583E58224D047
:1036F000F582E5833405F583E0045407FD75F00891
:10370000EEA42FF582E435F0F583E58224D0F5822E
:10371000E5833405F583EDF0E5702413F8E6FFE565
:10372000702412F8E675F008A42FF582E435F0F560
:1037300083E58224D0F582E5833405F583E0903F6C
:103740006093C454F04403FD7F02127F88E5702427
:1037500012F8E6FFE5702413F8E6FD7B401295DED3
:10376000E5702414F8E624F0FFE434FFFEEF78025D
:10377000C333CE33CED8F9FFE5702413F8E675F0E5
:1037800003A42430F582E43403F583E0FBA3E0FADC
:10379000A3E0F98F828E83120941E4FBFA797078F5
:1037A00041120344600E400CA870120A14BF80003E
:1037B00000023839E5702409F812098BE41203B1CC
:1037C000E4FBFA7980784B1202A77B0A7AD779A3B7
:1037D000783E12019E7B0A7AD7792378BE1200AD1B
:1037E000A8701209FC7B007A40791C7846E8C0E09A
:1037F000A87012098BD0E0F81202A77B007A247916
:1038000074784912019EA8701209FCE4FFFE7D7ACB
:103810007C44A8701209A312019EE4FBFAF9783FD8
:103820001200AD1203EFEC1203B1E4FBFA797A78DF
:10383000441202A7A8701209FCA87012098BECC0F0
:10384000E0EDC0E0EEC0E0EFC0E0E5702413F8E684
:1038500075F008A4FFE5702414F8E67C002FFFEC57
:1038600035F0FEEF7802C333CE33CED8F924F0F52D
:103870008274FF3EF583D0E0FFD0E0FED0E0FDD0C3
:10388000E0FC120A08A87012098BE5702415F8CB29
:10389000E6CB08E6FA08E6F91209717F0480067F94
:0538A0000080027F0121
:0738A500E5702418F5702204
:10AA540020202020557067726164696E6700202091
:10AA640020204669726D776172652E2E2E00245265
:0BAA740065763A203533323020240094
:0FA842000184FF4209B8FFFF4409C00000000075
:105E4600E47880F612ACE3C28575840F75E104E44C
:105E5600F5E275E344F58475B7B075840F758A83EA
:105E6600F597438901758D01758F01758E04F5428D
:105E7600F5430543E54370020542640F454270F25F
:105E8600438902E4F542F543AE42AF43E4FCFD7BB1
:105E9600507AC3F9F8D31208E7400FE58920E40ADF
:105EA6000543E54370E2054280DE759702129F1BAB
:105EB60012A1E38F41E4F584E541D39400400EE559
:105EC600EF5402D394004005AF4112799812AB45C6
:105ED600E4FF12AB6443EF04E4F542F5437D01AF02
:105EE6004312A99E0543E54370020542C39402E5A9
:105EF60042940040E8E4F520C22AC228C22EC22DF0
:105F0600C22C7880F6C22F08F67886F618F6788BBB
:105F1600F6F542F54374C82543F582E43409F58362
:105F2600E4F00543E54370020542B400E8E542B4F7
:105F360001E3E4F542F54374C82543F582E4340AE7
:105F4600F583E4F00543E5437002054264404542AB
:105F560070E5E4F584E5EF20E10CE5EF5408D39411
:105F6600004003D38001C392037D08E4FF12A5C558
:105F76007D087F0112A5C5128F5BE4788AF67882C8
:105F8600F6AB1CAA1DA91E7882E6FF75F020A4F5C3
:105F96008285F083120721FE788A26F6EE60057860
:105FA600820680DDEFD394004032AB1CAA1DA91EE9
:105FB60090000D120A88120708F541745512074E13
:105FC60012070864556002D22C74AA12074E1207F3
:105FD6000864AA6002D22CE54112074EE4F584E576
:105FE600EF5402D3940040047F018002E4FF128E36
:105FF600738F40E54020E036C22974FF788DF6089D
:10600600F608F608F67E007F107D007B007A0079A0
:1060160093120ADE7548FF754954754A84754B001C
:10602600754C107B007A00799312A5228002D22942
:1060360090AA79E493FF3395E0FEEF24D0FFEE3487
:10604600FFFE7C007D64120782AA06AB0790AA7841
:10605600E493FF3395E0FEEF24D0FFEE34FFFE7CA1
:10606600037DE8120782EF2BFBEE3AFA90AA7AE458
:1060760093FF3395E0FEEF24D0FFEE34FFFE7C0065
:106086007D0A120782EF2BFFEE3AFEA3E493FD335F
:1060960095E0FCED24D0FDEC34FFCD2F7892F6EDA3
:1060A6003E18F6E54030E103026154E4F542F5435B
:1060B600E543AE427805C333CE33CED8F9FFAB1CE9
:1060C600AA1DA91EF5828E831207216078E92FF991
:1060D600EA3EFA90000412072120E25EE4F53FE56D
:1060E6003FC37878965053E543AE427805C333CE26
:1060F60033CED8F9AB1CAA1DA91EF5828E831207D2
:1061060021FF7E00C006C0077D00E543AE4278054C
:10611600C333CE33CED8F929F9EA3EFA90000D12F0
:106126000A88788AE6853FF0A429F9EA35F0FAD09C
:1061360007D006120ADE053F80A50543E543700237
:1061460005420260B67F011284AFC22B8007E4FFCE
:106156001284AFD22BE4F542F5437A007B967D0399
:10616600AF43129B400543E54370020542C39402C8
:06617600E542940040E444
:01617C002200
:05AD4E00788BE6FF22F6
:0300230002884D03
:10884D00C0E0C0F0C083C082C0D075D000C000C0F1
:10885D0001C002C003C004C005C006C00730993E68
:10886D00C2997886067986E77881667015F67886DE
:01887D00F604
:0D887E0075270A75281300D528FCD527F6AC
:04888B00C285801C06
:0D888F0075271475281300D528FCD527F691
:10889C007886E624C8F582E4340AF583E0F599205D
:1088AC009803028948209A08202A05C29802894414
:1088BC00C29A7885E60624C8F582E43409F583E586
:1088CC0099F0C298E6FFB401129009C8E0FE70035B
:1088DC00F68069EE54072402788CF6EFB4020D781A
:1088EC008CE6B409079009C9E02403F67885E6FF05
:1088FC00B40007E4B40103F68042EFC3788C9640D1
:10890C003B7885E624FFFDE434FFFC7B017A097992
:10891C00C8129CEE7885E624C7F582E43409F58309
:08892C00E06F60047600801486
:0D89340075271475281300D528FCD527F6EB
:10894100121FDF78857600D007D006D005D004D07D
:1089510003D002D001D000D0D0D082D083D0F0D0CB
:02896100E03202
:100026009009C9E075F020A4AB1C251EF9E51D3525
:10003600F0FA90000D120A88788BE6FF18E68FF02A
:10004600A4252BF582E435F0F583120721FF7B000A
:040056007A0079298A
:10005A008F398B3A8A3B893CE4F584EA494B601C28
:10006A00AB3AAA3BA93C120708FFE539FD7C00120E
:0C007A00AD2FAB3AAA3BA93CEF12074E99
:0D008600753D14753E1300D53EFCD53DF6CA
:0E0093008539997F0112AA283099FDC2992261
:10A90100900AC87478F07885E624C7F582E43409A2
:09A91100F583E0900AC9F07F0211
:09A91A00E4F5847881EFF6D285A2
:0DA92300753914753A1300D53AFCD539F694
:07A93000900AC8E0F599222E
:10A74B00C9EFC9E964017028EDC39B40347878E602
:10A75B00FFEB2FFFE433FEEDC39FEE6480F87480B4
:10A76B0098501ED22AC3ED9B788BF6788776012200
:10A77B00B90214ED6B700AD22A788BF678877602C1
:08A78B0022C22AE47887F622BD
:10A2B600C9EFC9BAFF15BBFF12ED6B7002EC6A70ED
:10A2C60049D22A788BF67887E9F622E96401702567
:10A2D600C3ED9BEC9A401C7878E62BFFE43AFEC36C
:10A2E600ED9FEC9E500DD22AC3ED9B788BF67887B6
:10A2F6007601228015B90218ED6B7002EC6A700ABD
:10A30600D22A788BF67887760222C22AE47887F6F4
:01A316002224
:101FDF009009C8E0FF54F8F52AE4F584EF120AB827
:101FEF00202F09203C0A204F102058112069122061
:101FFF00801920961A20BB2020C428216029226234
:10200F0033229D3722CD3922E74122F24922FD4E5C
:10201F00233050237861222C70237098000023A85E
:10202F009009C9E0FD788EE6FB7F0180279009C9F2
:10203F00E0FCA3E0FD788DE6FA08E6FB7F01802B3C
:10204F00D22A788776030223A89009C9E0FD7890F9
:10205F00E6FB7F0212A74B0223A89009C9E0FCA35D
:10206F00E0FD788FE6FA08E6FB7F0212A2B60223A4
:10207F00A89009C9E0FD788EE6FB7F0112A74B20DF
:10208F002A030223A8801A9009C9E0FCA3E0FD7877
:10209F008DE6FA08E6FB7F0112A2B6202A0302237F
:1020AF00A8900AC87478F07F010223A5E4F584751F
:1020BF00EF100223A8C2ACE4F529D285FB7A007990
:1020CF00297F7F12005A7B007A0079297F1E120028
:1020DF005A7B007A0079297F0512005A7882E6121E
:1020EF000053788DE6120053788EE6120053788FE6
:1020FF00E61200537890E61200537891E6120053DF
:10210F007892E6120053E4F52B7493252BF8E61220
:10211F000053052BE52BC3941040EEE4F52B74B25E
:10212F00252BF582E43409F583E0120053052BE5E6
:10213F002BC3940640E87B007A007900AF29120088
:01214F005A35
:0D21500075370A75381300D538FCD537F601
:10215D000222179009C9E0FFC3788296400302223C
:10216D001EEF75F020A4251EF9E51D35F0851C34F4
:10217D00F5358936C2ACE4F529D285FB7A0079298B
:10218D007F7F12005A7B007A0079297F0D12005A49
:10219D00AB34AA35A936120708120053AB34AA3551
:1021AD00A936900001120050AB34AA35A936900023
:1021BD0002120050AB34AA35A9369000031200501C
:1021CD00AB34AA35A936900004120050E4F52BABC0
:1021DD0034E5362405F9E43535FA7E00E9252BF989
:1021ED00EE3AFA120708120053052BE52BC394089B
:0D21FD0040DD7B007A007900AF2912005A06
:0D220A0075370A75381300D538FCD537F646
:10221700C285D2AC0223A8900AC87478F0E4A3F070
:102227007F020223A512ACD078A31209FC900AC83A
:10223700747CF078A3E6A3F008E6A3F008E6A3F021
:1022470008E6A3F07C007D057B017A0A79C8129C19
:10225700EE900ACDEFF07F060223A59009C9E0FFB3
:10226700B4010FA3E0FDA3E0788DCDF608EDF602EB
:102277002370EFB4020A9009CAE0788DF602237042
:102287009009C9E0B4030CA3E0FFA3E0788FCFF671
:1022970008EFF6022370E4F52B9009C9E0FFE52B60
:1022A700C39F501B74CA252BF582E43409F583E0DC
:1022B700FF7493252BF8EFF6052BE52BB410DAE422
:1022C70078A2F60223707A007B327D01788BE6FFD5
:1022D700129B409009C9E0FDE4FF12A5C50223A89F
:1022E7009009C9E024FF92020223A89009C9E024BB
:1022F700FF92010223A87A007B327D017F00129BA7
:1023070040E4F52B74C9252BF582E43409F583E005
:10231700FF74BA252BF582E43409F583EFF0052B1A
:10232700E52BB406DFD22F8078788BE66005752D14
:1023370002800B202D05752D038003752D01900A52
:10234700C87479F0A3E52DF07C007D027B017A0A41
:1023570079C8129CEE900ACAEFF07F0312A91AE51A
:102367002D6401703CD22E8002D228788076F180CD
:10237700307A007B327D017F00129B40900AC8743F
:1023870079F09009C9E0900AC9F07C007D027B01D1
:102397007A0A79C8129CEE900ACAEFF07F0312A955
:1023A7001AE52A64A060030225B79009C8E064A172
:1023B70060030224A7A3E0C3788296400302249C0B
:1023C700AB1CAA1DA91EE0FF75F020A4F58285F0BD
:1023D70083120721F52DEF75F020A429F9EA35F0CE
:1023E700FA90000412072130E2379009C9E012ADD4
:1023F700498F2D900AC8747FF0A3E52DF02402FDC4
:10240700E433FC7B017A0A79C8129CEE74CA252D45
:10241700F582E4340AF583EFF0E52D2403FF022566
:10242700B49009C9E0FF12AD49C2ACE4F529D285E1
:10243700E52DD39406402B7B007A0079297F7F1204
:10244700005A7B007A007929AF2D12005AE4F52B48
:10245700E52BC3952D5007120026052B80F2052D7D
:102467008018E52D2478120053E4F52BE52BC3954E
:102477002D5007120026052B80F27B007A00790089
:05248700AF2912005A0C
:0D248C0075370A75381300D538FCD537F6C2
:102499000225A6900AC87478F07F010225B4900934
:1024A900C8E064A260030225B77882E6FFA3E0FED4
:1024B900C39F40030225ACA3E0FDC39F400302254F
:1024C900ACEE9D40030225AC9009C9E0F52BE4F57B
:1024D90032F5339009CAE0FFE52BD39F5026AF2B85
:1024E90012AD49AB1CAA1DA91E75F020E52BA4F558
:1024F9008285F0831207212533F533E43532F5322D
:10250900052B80CFC2ACE4F529D285FB7A00792965
:102519007F7F12005AC3E5339480E532940050025C
:102529008007E5324480120053AF331200549009FA
:10253900C9E0F52B9009CAE0FFE52BD39F5046E48B
:10254900F52CAB1CAA1DA91E75F020E52BA4F5825C
:1025590085F083120721FFE52CC39F5024E52B75D5
:10256900F020A429F9EA35F0FA90000D120A8878CA
:102579008BE6FF18E68FF0A4252C120049052C8064
:10258900C1052B80AF7B007A007900AF2912005A70
:0D25990075370A75381300D538FCD537F6B4
:1025A600C285D2AC800B900AC87478F07F0112A95C
:1025B6001AE52A6458704DFA7B327D01788BE6FF66
:1025C600129B40753C01753D0A753EC97B017A092F
:1025D60079C912A9CE8F2DE52D2478900AC8F0EF7F
:1025E6002401FDE433FC7B017A0A79C8129CEE745F
:1025F600C9252DF582E4340AF583EFF0E52D240292
:10260600FF12A91AE52A64806009E52A6488600336
:102616000227DC7887E6B4010F7A007B327D0178E9
:102626008BE6FF129B40801AE4F52BE52BC37878E6
:1026360096500F7A007B327D01AF2B129B40052B03
:1026460080E99009C8E05407F52DB4070A752C01F6
:10265600A3E0F52DA38006E4F52C9009C9E0F52E3C
:10266600152DE52EC378829640030227C9AB1CAA16
:102676001DA91E75F020E52EA4F58285F0831207AC
:1026860021FFE52DD39F40028F2D7887E6B40109FF
:10269600788BE6F531F5308009E4F5307878E61484
:1026A600F531788BA630788BE6D395314003022737
:1026B600A0E4F52BE52BC3952D4003022795E52EC7
:1026C60075F020A4AB1C251EF9E51D35F0FA900027
:1026D6000412072130E2030227909000011207211D
:1026E60064387041E52DD394044011E52C252B2444
:1026F600CAF582E43409F583E0FD80707885E6C387
:10270600952BFFE49400FE74C62FF58274093EF5FE
:1027160083E0FDE52E75F020A4AB1C251EF9E51D12
:1027260035F0FA8047AB1CAA1DA91E75F020E52ED0
:10273600A4F58285F083120721FF7885E6C39FFF03
:10274600E49400FE7C00EF252BFFEC3EFEEF252CEB
:10275600FFEC3EFE74C72FF58274093EF583E0FD5B
:10276600E52E75F020A429F9EA35F0FA90000D124D
:102776000A88788BE6FF18E68FF0A4FFE52B2FF585
:1027860082E435F0F583ED120760052B0226BAAF19
:102796002E12AC27788B060226AC788BA630E52E57
:1027A60075F020A4AB1C251EF9E51D35F0FA900046
:1027B6000412072130E5047884A62EE52A64887081
:1027C600158010E52EB4FF0E9009CAE0F520E52A23
:1027D600B4880312A901E52A64A8600302291478C3
:1027E60087E6B4010F7A007B327D01788BE6FF1213
:1027F6009B40801AE4F52BE52BC3787896500F7A28
:10280600007B327D01AF2B129B40052B80E990099E
:10281600C9E030E711547FFEA3E0FDEEF532EDF599
:1028260033752C03800C9009C9E0753200F53375B9
:102836002C0274C8252CF582E43409F583E0FF7474
:10284600C9252CF582E43409F583E0F52F8F2EE5B2
:102856002ED3952F4003022911E52EC37882964088
:102866000302290CAB1CAA1DA91E75F020E52EA497
:10287600F58285F083120721F52D7887E6B40109E4
:10288600788BE6F531F5308009E4F5307878E61492
:10289600F531788BA630788BE6D39531505EE4F52A
:1028A6002BE52BC3952D504AE52E75F020A4AB1CC5
:1028B600251EF9E51D35F0FA90000412072120E2E5
:1028C6002DE52C252B24CAF582E43409F583E0FD99
:1028D60090000D120A88788BE6FF18E68FF0A4FFA9
:1028E600E52B2FF582E435F0F583ED120760052B15
:1028F60080AFAF2E12AC27788B06809A788BA630E5
:0E290600E52D252CF52C052E02285512A901D1
:0129140022A0
:09A4760090001D12084AFFAEF02F
:10A47F008E418F429009B8E065417004A3E06542B8
:10A48F00603A9009A8740AF0E541A3F0E542A3F001
:10A49F007C007D037B017A0979A8129CEE9009ABB1
:10A4AF00EFF07B017A0979A87548017D047C0012D1
:0DA4BF009AAE9009B8E541F0A3E542F02205
:03A57400CCEECC5E
:10A577009009A8741AF0A3ECF0EFA3F07C007D0318
:10A587007B017A0979A8129CEE9009ABEFF07B0169
:10A597007A0979A87548017D047C00129AAE7B017F
:10A5A7007A0979A87D0A7C001292DAEF7002FF22FD
:0DA5B7009009A8E0647860037F00227F0116
:01A5C4002274
:10A9FB007A007B327D017F01129B4074FF9009B876
:10AA0B00F0A3F07F0A9009A8E4F0A3DFFC7B017AA6
:0DAA1B000979A87548017D0A7C00029AAEF9
:10872200E4F53FE53FC3788296400302884CE53F7B
:1087320075F020A4AB1C251EF9E51D35F0FA90005A
:108742000412072120E40302884712A4769009A8A4
:1087520074A1F0E53F75F020A4AB1C251EF9E51DC0
:1087620035F0FA90001F1207219009A9F07C007DD4
:10877200027B017A0979A8129CEE9009AAEFF07B9C
:10878200017A0979A8E4F5487D03FC129AAE7B01CF
:108792007A0979A87D647C001292DA8F40E540C3A1
:1087A20094025002804DE5402476FF9009A8E06FC4
:1087B2006002803FAB1CAA1DA91E75F020E53FA4F4
:1087C200F58285F083120721FFE54024FE6F6002E7
:1087D2008021E54024FFFDE434FFFC7B017A097926
:1087E200A8129CEE74A72540F582E43409F583E0D3
:1087F2006F6007AF3F12A9FB804BC2AFAB1CAA1D33
:10880200A91E75F020E53FA4F58285F083120721A9
:10881200FF7E00EEC0E0EFC0E0E53F75F020A42946
:10882200F9EA35F0FA90000D120A88C8E9C8CCEAD4
:10883200CCCDEBCD7B017A0979A9D0E0FFD0E0FE67
:0A8842001206E2D2AF053F028725BF
:01884C002209
:029E06008F3F8C
:109E0800EF75F020A4AB1C251EF9E51D35F0FA12FC
:109E1800A476AB1CAA1DA91E75F020E53FA4F58207
:109E280085F083120721F54024819009A8F0E53FC9
:109E380075F020A429F9EA35F0FA90001F120721DD
:109E48009009A9F0AF407E0090000D120A8878AA08
:109E58007C097D011206E2E5402402FDE433FC7B27
:109E6800017A0979A8129CEE74AA2540F582E43497
:109E780009F583EFF07B017A0979A8E5402403FD11
:099E8800E433FCE4F548029AAE53
:10A7020012ACBDC8ECC8C9EDC9CAEECACBEFCB903A
:10A7120009C0E0FCA3E0FDA3E0FEA3E0240AFFE4FD
:10A722003EFEE43DFDE43CFCD31208FD400C1287E2
:10A732002212ACBD9009C0120A087884E6FFF460C8
:09A7420007129E06788476FF22BE
:10F000007880E664F1600302F657E478ADF608F61E
:05F010007881E6601E9E
:0DF01500753F0A75401300D540FCD53FF64D
:10F0220078AE06E61870010678ADB627E108B6108C
:10F03200DDC2AF7584015398FC75FFDE75FFADE448
:10F0420078A9F618F6E4F584209830E478ADF6084D
:10F05200F6209823C378AEE6948818E694135017E6
:0DF06200753F0A75401300D540FCD53FF600
:10F06F0078AE06E61870DD0680DAB28680CD78A815
:10F07F00A699C298E6FF641A600302F15978ADF6BB
:10F08F0008F6209823C378AEE6948818E6941350B8
:01F09F001759
:0DF0A000753F0A75401300D540FCD53FF6C2
:10F0AD0078AE06E61870DD0680DA30988D78A9A660
:10F0BD0099C298E478ADF608F6209823C378AEE6A9
:08F0CD00948818E69413501713
:0DF0D500753F0A75401300D540FCD53FF68D
:10F0E20078AE06E61870DD0680DA20980302F04753
:10F0F20078A9A699C298E478ADF608F6209823C3B9
:0BF1020078AEE6948818E694135017CE
:0DF10D00753F0A75401300D540FCD53FF654
:10F11A0078AE06E61870DD0680DA20980302F0471A
:0AF12A0078A9A699C298D285C2996F
:0DF13400753F1475401300D540FCD53FF623
:06F141007599783099FD7C
:0DF14700753F0A75401300D540FCD53FF61A
:10F15400C28502F648EF6450600302F1EB78ADF625
:10F1640008F6209823C378AEE6948818E6941350E2
:01F174001783
:0DF17500753F0A75401300D540FCD53FF6EC
:10F1820078AE06E61870DD0680DA20980302F047B2
:0AF1920078A9A699C298D285C29907
:0DF19C00753F1475401300D540FCD53FF6BB
:08F1A9007599793099FDC299B6
:0DF1B100753F1475401300D540FCD53FF6A6
:08F1BE007599013099FDC29919
:0DF1C600753F1475401300D540FCD53FF691
:06F1D300E4F5993099FDFE
:0DF1D900753F0A75401300D540FCD53FF688
:10F1E600C28502F64878A8E6FF6401703ED285C261
:01F1F600997F
:0DF1F700753F1475401300D540FCD53FF660
:08F204007599783099FDC2995B
:0DF20C00753F1475401300D540FCD53FF64A
:06F21900E4F5993099FDB7
:0DF21F00753F0A75401300D540FCD53FF641
:10F22C00C28502F648EF6402600302F2FB78ADF689
:10F23C0008F6209823C378AEE6948818E694135009
:01F24C0017AA
:0DF24D00753F0A75401300D540FCD53FF613
:10F25A0078AE06E61870DD0680DA20980302F047D9
:10F26A0078A9A699C298E408F618E6FF13B392861D
:10F27A00EF25E0FEC3E49400EE94F0502DE6FD7F06
:10F28A000025E0FEC394E05021ED20E024E4F5845B
:10F29A0043B701758F0378AFEEF608EFF6F5828E65
:10F2AA0083E4F053B7F0F58F800478AA76FFE4F58B
:05F2BA0084D285C29919
:0DF2BF00753F1475401300D540FCD53FF697
:08F2CC007599783099FDC29993
:0DF2D400753F1475401300D540FCD53FF682
:08F2E10078AAE6F5993099FDC9
:0DF2E900753F0A75401300D540FCD53FF677
:10F2F600C28502F64878A8E66403600302F45678ED
:10F30600ADF608F6209823C378AEE6948818E694FE
:03F316001350177A
:0DF31900753F0A75401300D540FCD53FF646
:10F3260078AE06E61870DD0680DA20980302F0470C
:10F3360078A9A699C298E478ADF608F6209823C372
:0BF3460078AEE6948818E69413501788
:0DF35100753F0A75401300D540FCD53FF60E
:10F35E0078AE06E61870DD0680DA20980302F047D4
:10F36E0078ABA699C29878A9E6FF139286EF25E0AE
:10F37E00FEC3E49400EE94F0400302F047E67D00F5
:10F38E0025E0FCC394E0400302F047E4F58443B764
:10F39E0001758F0178ABE675F020A42DFFE5F03CEA
:10F3AE0078AFF608EFF6E4F58478ACF678ACE6C301
:10F3BE009420504CE408F608F6209823C378AEE665
:08F3CE00948818E6941350170F
:0DF3D600753F0A75401300D540FCD53FF689
:10F3E30078AE06E61870DD0680DA20980302F0474F
:10F3F30078AF0806E618CEE6CE70010614F5828EC5
:10F4030083E599F0C29878AC0680ACE4F58453B7F1
:09F41300F0F58FF584D285C29951
:0DF41C00753F1475401300D540FCD53FF638
:08F429007599783099FDC29934
:0DF43100753F1475401300D540FCD53FF623
:06F43E00E4F5993099FD90
:0DF44400753F0A75401300D540FCD53FF61A
:10F45100C28502F64878A8E6FD6404600302F5134C
:10F4610078ADF608F6209823C378AEE6948818E6BE
:04F471009413501789
:0DF47500753F0A75401300D540FCD53FF6E9
:10F4820078AE06E61870DD0680DA20980302F047AF
:10F4920078A9A699C298E625E078B1F608E4F6784C
:10F4A200AAF678ADF608F678B10806E618CEE6CEEA
:10F4B20070010614F5828E83E49378AA26F678AE5C
:10F4C20006E61870010678AEE6700418E66402706B
:05F4D200D6D285C299AD
:0DF4D700753F1475401300D540FCD53FF67D
:08F4E4007599783099FDC29979
:0DF4EC00753F1475401300D540FCD53FF668
:08F4F90078AAE6F5993099FDAF
:0DF50100753F0A75401300D540FCD53FF65C
:10F50E00C28502F648ED6405600302F63C78ADF65E
:10F51E0008F6209823C378AEE6948818E694135024
:01F52E0017C5
:0DF52F00753F0A75401300D540FCD53FF62E
:10F53C0078AE06E61870DD0680DA20980302F047F4
:10F54C0078A9A699C298E478ADF608F6209823C35A
:0BF55C0078AEE6948818E69413501770
:0DF56700753F0A75401300D540FCD53FF6F6
:10F5740078AE06E61870DD0680DA20980302F047BC
:0AF5840078ABA699C298D285C2990F
:0DF58E00753F1475401300D540FCD53FF6C5
:08F59B0075997F3099FDC299BA
:0DF5A300753F1475401300D540FCD53FF6B0
:10F5B0007599203099FD78A9E625E0FC78ABE675D1
:10F5C000F020A42400FFE5F03C78B1F608EFF6E463
:08F5D00078AAF678ACF6C299A6
:0DF5D800753F1475401300D540FCD53FF67B
:10F5E50078B1E6FE08E6F5828E83E493F5993099C5
:10F5F500FD78B10806E618CEE6CE70010614F58250
:10F605008E83E49378AA26F678AC06E6B420C2C2C7
:01F61500995B
:0DF61600753F1475401300D540FCD53FF63C
:08F6230078AAE6F5993099FD83
:0DF62B00753F0A75401300D540FCD53FF631
:10F63800C285800C78A8E6B40606E4F58475EF1058
:0FF6480078A8E66407600302F0477880F6D2AF37
:01F657002290
:10903F007F0012AA2820290B7A007B327D017F0046
:10904F00129B40302C0B7A007B1E7D017F00129B00
:10905F0040302817302D147A007B327D01788BE653
:10906F00FF129B40C22812970AD229202B0C302DB9
:10907F0009788076F112970AD22B302E2A302D27BD
:10908F00C22E12AD15E4FDFF12AC837BFF7AAA79D5
:10909F005412AAAA7D01E4FF12AC837BFF7AAA794E
:1090AF006212AAAA12F000302F0B7B017A0979BA4B
:1090BF0012A020C22F12ACBDC8ECC8C9EDC9CAEEB0
:1090CF00CACBEFCB9009C4120997EF245AFFE43EA5
:1090DF00FEE43DFDE43CFCD31208FD500F12ACBD85
:1090EF009009C41209B0D31208FD401212ACBD9002
:1090FF0009C4120A087B017A0979B21291FF202D57
:10910F001212ACBDE47B2C7A01F9F8C31208FD50A2
:04911F0002D22D2229
:0EAD0700125E4612903F12A702128D8280F556
:1085E9004D656D6F727920746573742E2E2E004D52
:1085F900656D6F7279206572726F722062616E6B40
:108609002025626400005EBCE2613FDD83C29C7E7E
:1086190020A3FD1F419DC3217FFCA2401E5F01E3F2
:10862900BD3E6082DC237D9FC1421CFEA0E1BF5D8F
:108639000380DE3C62BEE0025CDF81633D7C22C0D8
:108649009E1D43A1FF4618FAA427799BC584DA38F1
:1086590066E5BB5907DB856739BAE406581947A5AA
:10866900FB7826C49A653BD987045AB8E6A7F91B53
:1086790045C6987A24F8A6441A99C7257B3A648690
:10868900D85B05E7B98CD2306EEDB3510F4E10F2BD
:10869900AC2F7193CD114FADF3702ECC92D38D6F5A
:1086A90031B2EC0E50AFF1134DCE90722C6D33D127
:1086B9008F0C52B0EE326C8ED0530DEFB1F0AE4C40
:1086C9001291CF2D73CA947628ABF517490856B481
:1086D900EA6937D58B5709EBB536688AD495CB2922
:1086E90077F4AA4816E9B7550B88D6346A2B7597DB
:1086F900C94A14F6A8742AC896154BA9F7B6E80A08
:1087090054D7896B35000000002B6096CBDDEE0055
:098719002C96CBDDE5EEF7FAFD2C
:05A85100C1B101720A13
:10ACAA0074FFF51BF51AF519F518AF1BAE1AAD1995
:02ACBA00AC18D4
:01ACBC002275
:109CEE0015701570A870ECF608EDF6157015701558
:109CFE0070A870C6EBC608C6EAC608C6E9C6E57007
:049D0E0024FCF570CC
:109D1200F80808E4F6A870F608F6E5702407F9A832
:109D220070E6FE08E6FFC3099719E76480F8EE645F
:109D320080985037E5702404F8CBE6CB08E6FA08A1
:109D4200E6F98F828E83120721A870080866FFE564
:109D5200702403F8EFF6E690860E93A8700808F6D2
:109D6200A8700806E61870B20680AFA8700808E668
:019D7200FFF1
:079D7300E5702409F57022E0
:0BAD2F00ED6F78A7F6E690860E93FF0C
:01AD3A0022F6
:0300A30002A4CCE8
:10A4CC00C0E0C083C082C0D0E8C0E0EEC0E0EFC006
:10A4DC00E0E59830E1055398FDD231E59830E02461
:10A4EC007871E62401FFE433FEEF64404E70028085
:10A4FC00107871E606247EF582E4340BF583E59939
:10A50C00F05398FED0E0FFD0E0FED0E0F8D0D0D0F1
:06A51C0082D083D0E03282
:0A9AAE008B438A4489458C468D479E
:109AB800E47871F6758401D284E54824FF929BE42A
:109AC80078A8F678A8E6C39547E5466480F87480D8
:059AD800985060C2314E
:0D9ADD00754914754A1300D54AFCD549F6A9
:109AEA00E54724FFFFE54634FFFE78A8E66F7001DC
:109AFA00EE701EC2ACAB430545E545AA44700205AB
:109B0A004414F9120708F5993031FDC284D2AC80A9
:109B1A0016AB430545E545AA447002054414F912FB
:109B2A000708F5993031FD7F0112AA2878A8068026
:059B3A0090C284AF475A
:019B3F002203
:0A92DA008B418A4289438C448D4584
:1092E40012ACBD78A91209FCE478A8F612ACBDEC66
:1092F400C0E0EDC0E0EEC0E0EFC0E078A912098B59
:10930400CBEFCBCAEECAC9EDC9C8ECC8D0E0FFD0D8
:10931400E0FED0E0FDD0E0FCC3EF9BFFEE9AFEED53
:1093240099FDEC98FCE47B01FAF9F8C31208FD50AE
:10933400037F00227871E6FED394004053900B7EA5
:10934400E0FDB478037F0122ED54F8647860037F74
:109354000022900B7EE05407240278A8F66E703049
:109364007871E6D39545E5446480F87480984006A6
:10937400AE44AF4580067871E6FF7E00A843AC4258
:10938400AD417B017A0B797E1206E278A8E6FF22D2
:089394007F0112AA280292F0E9
:07AD4200E47871F6D2312222
:10A5C500EF7025F5847598D0F584759115F584752A
:10A5D500C90875CBFFED90870D93F5CA75C804E4DE
:10A5E500F584D2ACC2BC80267584017598D0E4F59B
:10A5F50084E589540F4420F589758E02ED908717FF
:10A6050093F58DD28E43E74043F74012AD42D2AF6A
:01A615002222
:10A17800900BBE120A2D00000000900BC2120A2D8F
:10A1880000000000900B757464F0E478A8F678A8D5
:10A19800E6FFC394025043EF25E025E02476F582DC
:10A1A800E4340BF583E4F0EF25E025E02477F5822D
:10A1B800E4340BF583E4F0EF25E025E02478F5821C
:10A1C800E4340BF583E4F0EF25E025E02479F5820B
:0AA1D800E4340BF583E4F00680B4D4
:01A1E200225A
:10AB4500D2AFD2A9C2BBE4F584E589540F4401F51F
:0FAB550089758E02758CAFE4F58AD28C02A178D7
:028C900015705D
:108C9200A870E4F6A870E6FFC394024003028D7F39
:108CA200EF25E025E02479F582E4340BF583E0FF3B
:108CB200D394005003028D54E625E025E02477F595
:108CC20082E4340BF583E06003028D54EF30E01947
:108CD200E6FF25E025E02479F582E4340BF583E014
:108CE200D3940140047D0080067D01A870E6FF1246
:108CF200A10AA870E6FF25E025E02479F582E43494
:108D02000BF583E0B401057D0112A10AA870E6FF0C
:108D120025E025E02479F582E4340BF583E014F0B4
:108D2200EF25E025E02479F582E4340BF583E06059
:108D320021E6FF25E025E02478F582E4340BF58373
:108D4200E0FEEF25E025E02477F582E4340BF5839D
:108D5200EEF0A870E6FF25E025E02477F582E43402
:108D62000BF583E06011EF25E025E02477F582E43E
:0D8D7200340BF583E014F0A87006028C9617
:038D7F000570225A
:03000B00029981D6
:10998100C0E0C0F0C083C082C0D0E8C0E0E9C0E060
:10999100EAC0E0EBC0E0ECC0E0EDC0E0EEC0E0EF1B
:1099A100C0E0758CAF900BBEE0FCA3E0FDA3E0FE30
:1099B100A3E02401FFE43EFEE43DFDE43CFC900B0A
:1099C100BE120A08900B75E014F0E07025900BC2EE
:1099D100E0FCA3E0FDA3E0FEA3E02401FFE43EFEE2
:1099E100E43DFDE43CFC900BC2120A08900B757437
:1099F10064F0128C9012AB23D0E0FFD0E0FED0E0F7
:109A0100FDD0E0FCD0E0FBD0E0FAD0E0F9D0E0F806
:0B9A1100D0D0D082D083D0F0D0E03263
:10A99E001570A870EDF61570A870EFF6A870E6FFAA
:10A9AE00C39402501608E6FDEF25E025E02476F567
:10A9BE0082E4340BF583EDF012A10A0570057022C6
:109B400015701570A870EAF608EBF61570A870EDA0
:109B5000F61570A870EFF6A870E6FFC39402506A7D
:109B6000EF25E025E02479F582E4340BF583E070FD
:109B700059E6FB25E025E02477F582E4340BF583F4
:109B8000E0704708E625E004FFA870E6FA25E02526
:109B9000E02479F582E4340BF583EFF00808E6FE63
:109BA00008E6FF7C007D0A1207E9EA25E025E024AB
:109BB00078F582E4340BF583EFF0EB25E025E02423
:109BC00077F582E4340BF583E4F0E5702404F57056
:019BD0002272
:0EA10A001570A870EDF61570A870EFF61570C0
:10A11800A87008E6FFC394025024EF25E025E02448
:10A1280076F582E4340BF583E06013A8700808E63E
:10A1380070047F0180027F00A8700808EFF6A870FD
:10A14800A68475840FA87008E6FF700BA87008082D
:10A15800E624FF9286800DEFB40109A8700808E68E
:09A1680024FF9287A870E6F5843B
:07A171000570057005702266
:10ACBD00C2AF900BBEE0FCA3E0FDA3E0FEA3E0FF5E
:02ACCD00D2AF04
:01ACCF002262
:10ACD000C2AF900BC2E0FCA3E0FDA3E0FEA3E0FF47
:02ACE000D2AFF1
:01ACE200224F
:10AA28001570A870EFF6A870E670057873F608F64A
:10AA38003030167872E675F064A4FFC37874E69F28
:0CAA480018E695F0500375FFA50570227C
:10AB6400D230E47873F608F6EF78726003F6800268
:0FAB7400760A75FF0775FFA5E4F58475EF0422D7
:10ACE300C230E47873F608F6787276FF75FFDE7586
:03ACF300FFAD2290
:10AB2300787406E6187001063030167872E675F010
:10AB330064A4FFC37874E69F18E695F0500375FF8D
:02AB4300A52249
:04AA7F008E448F452D
:10AA8300E4F546F547C3E5479545E5469544501635
:10AA93007FE87E0312A36F7F0112AA280547E547CB
:06AAA30070E3054680DFB0
:01AAA900228A
:04A36F008E648F6504
:10A37300D3E56594FAE56494005010AF65EFD39488
:10A383000040407E1600DEFD1F80F2856466856511
:10A3930067D3E56794FAE566940040157FFA7E007B
:10A3A30012A36F74062567F56774FF3566F566803B
:10A3B300E0D3E5659400E56494004007AF67AE66BB
:03A3C30012A36F73
:01A3C6002274
:10A24E0075500075510075524A7B007A0079487D31
:01A25E0002FD
:08A25F008B4C8A4D894E8D4F96
:10A267007F0112AA28AB50AA51A95212081F240035
:10A27700FFE5F034E0FE854C53854D54854E55E49B
:10A28700FDEDC3954F501BEF2DF582E43EF583E4BA
:10A2970093AB53AA54A9558D827583001207600D9D
:0FA2A70080DFAB50AA51A952E4854FF002088224
:10945D00754112754234754900754A00754B437B51
:07946D00007A0079417D0245
:089474008B458A4689478D48AB
:10947C007880E664F1600302951112ACE3C2AFE4AC
:10948C00F58443B701758F01AB49AA4AA94B120861
:10949C001F2400FFE5F034E078A8F608EFF6AA46A2
:1094AC00A94778ACA64508C6EAC608C6E9C6E4785A
:1094BC00AAF678AAE6C39548503278ACCBE6CB082E
:1094CC000806E618CAE6CA70010614F912070878ED
:1094DC00ABF6E6FF78A80806E618CCE6CC700106D9
:1094EC0014F5828C83EFF078AA0680C6E4F58F53CE
:1094FC00B7F0AB49AA4AA94B8548F0120882D2AF03
:05950C00E4FF12AB6456
:019511002237
:10A6B4007880E664F17046C2AF12ACE3E4F58443FB
:10A6C400B701758F0378A976E008F678A8F678A91B
:10A6D400E6FE08E6F5828E83E4F07F0112AA28786C
:10A6E400AAE426F618740236F61806E6C39408405F
:0DA6F400DDE4F58F53B7F0D2AFFF12AB6479
:01A701002235
:10970A0012A6B4E4F543F544F549754A00754B438E
:10971A00FB7A00798D7D1612947412945DE4F540FB
:10972A00E540C37878965073E4F53FAB1CAA1DA9AF
:10973A001E75F020E53FA4F58285F08312072160AB
:10974A0056E53F75F020A429F9EA35F0FA90000DA4
:10975A00120A88788AE68540F0A429F9EA35F0FAEF
:10976A00EBC0E0EAC0E0E9C0E0AB1CAA1DA91E7587
:10977A00F020E53FA4F58285F083120721FD7549A3
:10978A0000754A00754B43D0E0F9D0E0FAD0E0FB0F
:10979A00129474053F80940540808512945DE478A4
:0297AA0080F647
:0197AC00229A
:028E73008F442A
:108E7500E4F54AF54BF547F55075510075524AFB37
:108E85007A00798D7D1612A25F12A24EE5496434EF
:108E95007004E54864127003434701E4F546E5466E
:108EA500C37878964003028F46E4F545AB1CAA1DAE
:108EB500A91E75F020E545A4F58285F083120721EA
:108EC500607AE5446054E54575F020A429F9EA3552
:108ED500F0FA90000D120A88788AE68546F0A429F2
:108EE500F9EA35F0FAEBC0E0EAC0E0E9C0E0AB1C16
:108EF500AA1DA91E75F020E545A4F58285F083120B
:108F05000721FD75500075510075524AD0E0F9D022
:108F1500E0FAD0E0FB12A25F801DAB1CAA1DA91EC2
:108F250075F020E545A4F58285F083120721254BD0
:108F3500F54BE4354AF54A0545028EB10546028EE4
:108F4500A312A24EE54964347004E5486412700327
:058F5500434702AF4795
:018F5A0022F4
:10ABA100EF540778AAF6EF30E306E64420F6800476
:0CABB10078AAE6F678AAE644C0F6F5C8DB
:01ABBD002275
:027998008F441A
:10799A0012AD157D017F0212AC837BFF7A8579E9EE
:1079AA00124EF6E478A9F612ACE3C2AFE478A8F670
:1079BA0078A8E6FFC395444003027AFB12ABA1788C
:1079CA00A8E6FF7D0312AC837FDA12AC6D9020002B
:1079DA00AF82AE83C3EF94FFEE94FF5005E4F0A3A9
:1079EA0080EE902000AF82AE83C3EF94FFEE94FF47
:1079FA00500CE0600678A976018003A380E778A995
:107A0A00E66003027AFB78A8E6FF7D0312AC837F67
:107A1A00D912AC6D902000AF82AE83C3EF94FFEE13
:107A2A0094FF50067455F0A380ED902000AF82AE0B
:107A3A0083C3EF94FFEE94FF500EE064556006781E
:107A4A00A976018003A380E578A9E66003027AFBA0
:107A5A0078A8E6FF7D0312AC837FD812AC6D902024
:107A6A0000AF82AE83C3EF94FFEE94FF500674AA70
:107A7A00F0A380ED902000AF82AE83C3EF94FFEEB7
:107A8A0094FF500EE064AA600678A976018003A3E9
:107A9A0080E578A9E6705A78A8E6FF7D0312AC83E0
:107AAA007FD712AC6D902000AF82AE83C3EF94FFF4
:107ABA00EE94FF500674FFF0A380ED902000AF8291
:107ACA00AE83C3EF94FFEE94FF500DE0F4600678A6
:107ADA00A976018003A380E678A9E6701478A8E65F
:107AEA00FF7D0312AC837FD612AC6D78A8060279AB
:107AFA00BAD2AFE4FF12AB6412ABA178A9E6601B5D
:107B0A007D02E412AC837BFF7A8579F878A8E6F5E2
:0B7B1A0048124EF67F0012AA2880F9E6
:017B2500223D
:10A1E300E4F58475A338F5A275A10475840F759CF5
:10A1F300FF759DFF759EFF759FFF75F8FF75E8FF5F
:10A2030075D8FF75C8FFFF12ABA1902000E078A8B6
:10A21300F67455F0E064556008E6F0E4F584F5A3C0
:10A223002278A8E6F07F0812ABA1E078A8F674AA1A
:10A23300F0E0B4AA0AE6F0E4FF12ABA17F102278A3
:0AA24300A8E6F0E4FF12ABA17F08CB
:01A24D0022EE
:029666008F6211
:1096680020320302970943A0F075840F43A60FC266
:1096780090C294D2957F017E0012A36FD296E4F532
:10968800637F0A7E0012A36F30A7090563E563C3F1
:1096980094C840EDC2967F017E0012A36FC295D296
:1096A8009075840F75A6FF7F017E0012A36FE56297
:1096B80054F0FFE5A054014FF5A0A21E92947F013B
:1096C8007E0012A36FD2967F017E0012A36FC2960E
:1096D8007F017E0012A36FE562C454F0FFE5A05439
:1096E800014FF5A0A21E92947F017E0012A36FD2B3
:1096F800967F017E0012A36FC2967F017E0012A39F
:019708006FF1
:01970900223D
:10A7DA008F4453A00FE54454F042A0D2967F017EE5
:10A7EA000012A36FC2967F017E0012A36F53A00FBF
:10A7FA00E544C454F042A0D2967F017E0012A36FB2
:10A80A00C2967F017E0012A36F7F647E0002A36F4F
:109F1B00E478A8F608F6C296C295C29475840F75BC
:109F2B00A6FF43A503D290D29153A00143A020D208
:109F3B00967F01FE12A36FC2967F017E0012AA7F4D
:109F4B007F2012A7DA43A0F075840F43A60FC290AF
:109F5B00C294D2957F017E0012A36FD2967F647E4E
:109F6B000012A36F30A703C23222D232C21E7F244B
:109F7B00129666C21E7F0B129666C21E7F20129629
:109F8B0066C21E7F0C129666C21E7F01129666C2B7
:069F9B001E7F061296660F
:019FA100229D
:0DAD1500C21E7F01129666E4FDFF02AC83B2
:10ACF600EF6006C21E7F0F8004C21E7F0C1296668E
:01AD0600222A
:10AC8300ED5403C43354E0FEEF541F44804EFFC21F
:04AC93001E029666A1
:10AC6D008F61E561640D600BE561640A6005D21EBC
:06AC7D00129666AF612291
:10AAFC008B688A69896AAB68AA69A96A12070860B7
:10AB0C0015056AE56A7002056914F9120708FFD287
:07AB1C001E12966680E02284
:1000A60002045BE86480F8E933E83360110460F029
:1000B600ED33EC337009E8FCE9FDEAFEEBFF2204C0
:1000C60060DED3EB9FEA9EE99DE8C2E78CF0C2F7BB
:1000D60095F0400CE8CCF8E9CDF9EACEFAEBCFFB87
:1000E60012042685D0F05804700320D5B3E80470B6
:1000F600075002B2D502046592D5EC0460F7E4CC51
:10010600C0E0C398F8603B94186008400DD0E0FB4F
:1001160002043DE4FBFAC9FC8028E830E406E4C9A1
:10012600FBE4CAFCE830E305E4C9CACBFCE85407A3
:100136006010F8C3E913F9EA13FAEB13FBEC13FCAE
:10014600D8F130F52FC3E49CFCEF9BFFEE9AFEED51
:1001560099FDD0E0FBEF4E4D4C701222DB030204FA
:1001660062EC2CFCEF33FFEE33FEED33FDED30E7B2
:10017600EB02043DEF2BFFEE3AFEED39FDD0E0FB3E
:1001860050130BBB0003020465ED13FDEE13FEEFE7
:0801960013FFEC13FC02043D11
:10019E00EC4D6011E8497017ED33EC3304600DE45B
:1001AE00FCFFFEFD22E933E8330470F802045B1213
:1001BE00042658046009E4CC248150062850090214
:1001CE000465284003020462C0E0EB4A7044B98023
:1001DE0006D0E0FB020451EF4E701CBD8008EBFF11
:1001EE00EAFEE9FD80EBE98DF0A4FEE5F002028760
:1001FE00E9CDF9EAFEEBFFEF89F0A4FCE5F0CE893C
:10020E00F0A42EFFE435F0CD89F0A42DFEE435F0F8
:10021E008067EF4E7005BD80D780C3EF8BF0A4AC26
:10022E00F0EE8BF0A42CFCE435F0F8EF8AF0A42C61
:10023E00E5F038FCE433CB8DF0A42CFCE5F03BF874
:10024E00EE8AF0A42CFCE5F038F8E433CF89F0A464
:10025E002CFCE5F038CF3400CE89F0A42FFFE5F06A
:10026E003EFEE433C98DF0A42EFEE5F039CD8AF0C2
:10027E00A42FFFE5F03EFEE43DFD33D0E0FB50073A
:10028E000BBB000F020465EC2CFCEF33FFEE33FECC
:06029E00ED33FD02043DFA
:1002A400020465EC5D046005E85904700302045B14
:1002B400120426580460F6EC4860F2EC7004FDFE6B
:1002C400FF22C860DB2481C85009C398600250062D
:1002D4000204629850CAF582E9294B4A7005AB8240
:1002E40002045175F0007C1A7880C3EF9BEE9AEDFE
:1002F40099400DC3EF9BFFEE9AFEED99FDE842F0A5
:10030400DC23ACF0D0E0FFD0E0FED0E0FDAB8220F7
:10031400E7101BEB60BAEC2CFCEF33FFEE33FEED81
:1003240033FD02043DE803F830E705C0F075F00042
:10033400EF2FFFEE33FEED33FD40B830E7C280AA65
:1003440074F8CC6480CCC86480C8F582046043C36C
:10035400EB9FF5F0EA9E42F0E99D42F0E89C45F0FF
:1003640060305018E5825FFFE582F42B5582FB5024
:10037400210ABA001D09B90019088016E5825BFB41
:10038400E582F42F5582FF50090EBE00050DBD0015
:10039400010CC3EB9FF5F0EA9E42F0E99D42F0E8C0
:0D03A4009C45F06007CC4820E701B3EC2237
:1003B10075F020800E75F010800575F0087D007EC7
:1003C100007F003392D530D5031208D9EC334010A9
:1003D100EF33FFEE33FEED33FDEC33FCD5F0ED22D0
:0E03E100E5F0247EA2D513CC92E7CDCEFF220C
:1003EF00EDD2E7CD33EC3392D524814006E4FFFE06
:1003FF00FDFC22FCE4CFCECDCC24E0501174FF8065
:10040F00EDC3CC13CCCD13CDCE13CECF13CF047001
:07041F00F030D5DE0208D920
:104E9400E55C2448F8E6055C227845301C02784835
:104EA400E475F001120A780207082015EB7F2ED270
:104EB400158018EF540F2490D43440D4FF30190BCC
:104EC400EF24BFB41A0050032461FFE55D600215AE
:104ED4005D0560E5607002055F301C0D7845E47582
:104EE400F001120A78EF02074E02AC6D7403D21C73
:104EF4008003E4C21CF55C8B458A468947E4F55D72
:104F0400F55FF560E55D60077F20124ECF80F57593
:104F14005EFFC216C215C217C218C21AC21BC21D36
:104F2400124E9DFF700D301C057F00124EE0AF60E5
:104F3400AE5F22B4255FC2D5C219124E9DFF24D0A4
:104F4400B40A00501A75F00A785D30D50508B6FF2A
:104F54000106C6A426F620D5047002D21880D924EE
:104F6400CFB41A00EF5004C2E5D2190251CDD216C3
:104F740080C6D21580C0D21780BCD2D580BAD21ACE
:104F840080B47F20124ECF2017077401B55D004016
:104F9400F1124E94FF124ECF024F08D21DD21B8045
:104FA40095124E94FB124E94FA124E94F94A4B7099
:104FB4000679C47A527BFF20172EE55D602A7E00B5
:104FC4008E8275830012072160060EEE655E70F016
:104FD400C2D5EBC0E0EAC0E0E9C0E0EE12522DD049
:104FE400E0F9D0E0FAD0E0FB120708FF60AAEBC0BA
:104FF400E0EAC0E0E9C0E0124ECFD0E02401F9D0ED
:10500400E03400FAD0E0FBE55E0460DCD55ED980D4
:1050140087D21780A212521060F7E55E7001041265
:105024000470A95E600DE55E600914F55E1252B766
:10503400EF60F3EA30E702F404C3995077EAF42509
:105044005E0430E701E404F55E800D12521060C185
:10505400EA055E255E120470EA785BF630E701E447
:10506400255E04D55E04201A011412522DE4C0E01A
:105074001252B7785BE6601320E70714F6124EB7B6
:10508400802204F6D0E014C0E07F00124EB7E55E43
:105094006007124EAE155E800B301A03124EAED06E
:1050A400E0024F08D0E00480C512521060A0E55E13
:1050B40004120470785BEAF6E55E201A02600104CB
:0550C400240412522D2E
:1050C90074FF04C0E01252B7124EB7E55E201A020F
:1050D9006003124EAED0E0B55EE87F45124EC1784E
:1050E9005BE67F2B30E7047F2DF404C0E0124ECF3E
:1050F900D0E075F00A84C0F0124EB8D0E0124EB874
:10510900024F08791080027908C21BC21D8008D29B
:10511900D5790A8004790AC2D5E55E047002F55E84
:10512900E4FAFDFEFF124E94FC7B08201613124E82
:1051390094FD7B1030150A124E94FE124E94FF7B9B
:1051490020EC3382D592D55013C3E43015069FFF66
:10515900E49EFEE42016039DFDE49CFCE4CBF8C22A
:1051690016EC700CCFCECDCCE824F8F870F380178C
:10517900C3EF33FFEE33FEED33FDEC33FCEB33FBD2
:10518900994002FB0FD8E9EB301605F8D0E0C44886
:10519900B216C0E00AEC4D4E4F78207B0070C2EA8F
:1051A900B55E0040BCC0E012522FD0F0D0E020160E
:1051B90004C4C0E0C4B216C0F0124EB8D0F0D5F0A5
:1051C900EB024F08120AB84FA553510C584F764CB1
:1051D9004F724251104F5118445118494F8B435146
:1051E9001E55504F4650AD4550194752E4504F7A1D
:1051F9002D4F7E2E4FA12B4F82234F9F2052CD2A18
:105209004F3A4800004F99E55EB4FF03755E0612F8
:105219004E94FC124E94FD124E94FE124E94FF7859
:105229005402049F790AA2D5201814301A09B9101A
:10523900020404B9080104A2D5201B02500104206C
:1052490017689217B55D005034C0E07F20301819F7
:105259007F30A217721B721A500F125286C217C2E0
:105269001BC21AC21D7F30800F301A03E9C0E01239
:105279004ECF301A03D0E0F9D0E0B55DCC301A1723
:105289007F30B9100C124ECF7F583019077F7880C4
:1052990003B90803124ECF3017057F2D024ECF7F79
:1052A90020201DF87F2B201BF322921780CF7F002F
:1052B900B4070050052454F8E6FF22286E756C6C7B
:1052C9002900D216124E943016F8C216785D30D5E0
:1052D9000108F6024F3A2D50434958124E942403BF
:1052E900B405004001E49052DF93124EC0743A12A3
:0A52F9004EC0D218755D0402510C7E
:0DAD2200ED33EC3360065004EC6480FC223D
:109512008F478E468D458C4474FFFFFEFDFCAB47A2
:10952200AA46A945A844C31208FD602C7F807E96F6
:109532007D187C4BAB47AA46A945A8441203446058
:109542000250157F807E967D187CCBAB47AA46A938
:1095520045A8441203445009AF47AE46AD45AC445A
:1095620022AF47AE46AD45AC441203EF8F4B8E4A55
:109572008D498C48EC1203B1C8ECC8C9EDC9CAEEDA
:10958200CACBEFCBAF47AE46AD45AC441200A9E41F
:10959200FBFAF9F8120344601A401874FF254BF5E0
:1095A2004BE54A34FFF54AE54934FFF549E54834CD
:1095B200FFF548AF4BAE4AAD49AC48EC1203B122BD
:10042600E9D2E7C933E833F892D5EDD2E7CD33EC1C
:0704360033FC5002B2D52295
:10043D00EC30E7100FBF000C0EBE00080DBD000420
:10044D000BEB6014A2D5EB13FCED92E7FD2274FFCC
:10045D00FCFDFEFF22E480F8A2D574FF13FC7D8025
:03046D00E480EF39
:10047000F920E72824F950037907E4F42402FB1853
:10048000DBFDE624FB5014E9600DE4F618E604F603
:0F049000B40A08E4F6D9F57401F60A22C2D5229F
:10049F00ED33EC3392D5FA602AB4FF33EDC2E77B2C
:1004AF00FF60067A0479C4E4227A0479CD20D5045A
:1004BF007A0479C8224E614E002B494E46002D49D1
:1004CF004E4600E47A08F608DAFC7B00740722E84F
:1004DF00C0E0ECC0E0EDC0E0EEC0E0EFC0E0EA75D8
:1004EF00F010A4CAABF075F04DA42BFBE435F0FC73
:1004FF00EA2410FAEB34C5FBEC34D9FCEDC2E7FF6C
:10050F0075F056A4F42411C5F0F434C58FF0A42A65
:10051F00E5F03BE43CF620E7141205D2D0E0FFD023
:10052F00E0FED0E0FDD0E0FC1202A78014F404122C
:10053F0005D2D0E0FFD0E0FED0E0FDD0E0FC12010C
:10054F009ED0E0F8E6FAEDD2E7CD33EC332482FB10
:10055F00E4C3CF33CFCE33CECD33CD33DBF37B07F5
:10056F0075F00A846004F6081B0AE5F0F6088FF0B0
:10057F00740AA4FFACF08EF0740AA42CFEACF050F9
:10058F00010C8DF0740AA42CFDE435F0F608DBDEC7
:03059F00740722BC
:1005A2003F8000004120000042C80000447A000061
:1005B200461C400047C35000497424004B189680E3
:1005C2004CBEBC205A0E1BCA6753C21C749DC5AEDA
:1005D200FB60065407601C2323120600EB543860AC
:1005E200091205EC1205FB12019EECF8EDF9EEFA88
:1005F200EFCB22EB1205FB80F1543803241C90054B
:10060200A2FE93FC0EEE93FD0EEE930ECE93FF220E
:03000000029D7AE4
:0C9D7A00787FE4F6D8FD7581B2029DC12F
:10061200E709F608DFFA8046E709F208DFFA803ECA
:1006220088828C83E709F0A3DFFA8032E309F608B7
:10063200DFFA8078E309F208DFFA807088828C831F
:10064200E309F0A3DFFA806489828A83E0A3F608D3
:10065200DFFA805889828A83E0A3F208DFFA804CAD
:1006620080D280FA80C680D4806980F28033801084
:1006720080A680EA809A80A880DA80E280CA8033ED
:1006820089828A83ECFAE493A3C8C582C8CCC58365
:10069200CCF0A3C8C582C8CCC583CCDFE9DEE78035
:1006A2000D89828A83E493A3F608DFF9ECFAA9F0B4
:1006B200EDFB2289828A83ECFAE0A3C8C582C8CC0A
:1006C200C583CCF0A3C8C582C8CCC583CCDFEADE23
:1006D200E880DB89828A83E493A3F208DFF980CC85
:1006E20088F0EF60010E4E60C388F0ED2402B4047E
:1006F2000050B9F582EB2402B4040050AF23234525
:06070200822390066273E1
:10070800BB010689828A83E0225002E722BBFE02EF
:09071800E32289828A83E4932222
:10072100BB010CE58229F582E5833AF583E022508D
:1007310006E92582F8E622BBFE06E92582F8E222D7
:0D074100E58229F582E5833AF583E49322F1
:10074E00BB010689828A83F0225002F722BBFE018A
:02075E00F32284
:10076000F8BB010DE58229F582E5833AF583E8F0CF
:10077000225006E92582C8F622BBFE05E92582C87B
:02078000F22263
:10078200EF8DF0A4A8F0CF8CF0A428CE8DF0A42E8B
:02079200FE2245
:10079400BC000BBE0029EF8DF084FFADF022E4CC49
:1007A400F875F008EF2FFFEE33FEEC33FCEE9DEC12
:1007B400984005FCEE9DFE0FD5F0E9E4CEFD22ED58
:1007C400F8F5F0EE8420D21CFEADF075F008EF2FA2
:1007D400FFED33FD4007985006D5F0F222C398FD93
:0507E4000FD5F0EA2230
:1007E900C2D5EC30E709B2D5E4C39DFDE49CFCEE2B
:1007F90030E715B2D5E4C39FFFE49EFE120794C308
:10080900E49DFDE49CFC800312079430D507C3E402
:060819009FFFE49EFE2299
:10081F00BB010A89828A83E0F5F0A3E022500687A4
:10082F00F009E71922BBFE07E3F5F009E319228966
:0B083F00828A83E493F5F07401932299
:10084A00BB0110E58229F582E5833AF583E0F5F0EC
:10085A00A3E0225009E92582F886F008E622BBFEC9
:10086A000AE92582F8E2F5F008E222E5832AF5830F
:08087A00E993F5F0A3E99322D4
:10088200BB010789828A83020B0A500B09C5F02734
:10089200F7C5F01937F722BBFE0D09F8E325F0F38F
:1008A200C5F019E338F322F889828A83740193250B
:0808B200F0C5F0F8E4933822D0
:1008BA00BB010A89828A83F0E5F0A3F0225006F789
:0F08CA0009A7F01922BBFE06F3E5F009F3192286
:0E08D900C3E49FFFE49EFEE49DFDE49CFC2230
:1008E700EB9FF5F0EA9E42F0E99D42F0EC6480C888
:0608F70064809845F02228
:1008FD00EB9FF5F0EA9E42F0E99D42F0E89C45F051
:01090D0022C7
:10090E00E8600FEFC333FFEE33FEED33FDEC33FC47
:03091E00D8F122EB
:10092100BB010789828A830209975005E9F8020908
:100931008BBBFE05E9F8020B2089828A83020B2C0E
:10094100BB010DE58229F582E5833AF5830209971A
:100951005007E92582F802098BBBFE07E92582F8D9
:10096100020B20E58229F582E5833AF583020B2CFF
:10097100BB010789828A83020A085005E9F8020946
:0A098100FCBBFE05E9F8020B492259
:0C098B00E6FC08E6FD08E6FE08E6FF2298
:0C099700E0FCA3E0FDA3E0FEA3E0FF22D3
:0D09A300E6FB08E6F908E6FA08E6CBF822C4
:0C09B000E0F8A3E0F9A3E0FAA3E0FB22CA
:1009BC00E493F8740193F9740293FA740393FB2291
:1009CC00BB010DE58229F582E5833AF5830209B076
:1009DC005007E92582F80209A3BBFE07E92582F836
:1009EC00020B3CE58229F582E5833AF5830209BCCA
:0C09FC00ECF608EDF608EEF608EFF62227
:0C0A0800ECF0A3EDF0A3EEF0A3EFF02261
:100A1400D083D082E493F608740193F608740293A9
:090A2400F608740393F6740473E0
:100A2D00A8828583F0D083D082120A44120A441220
:100A3D000A44120A44E473E493A3C583C5F0C58345
:100A4D00C8C582C8F0A3C583C5F0C583C8C582C813
:010A5D002276
:100A5E00BB010789828A83020A2D5005E9F8020A32
:0A0A6E0014BBFE05E9F8020B552247
:100A7800FAE6FB0808E6F925F0F618E6CA3AF6227F
:100A8800BB010DE58229F582E5833AF583020B77F0
:100A98005007E92582F8020B6EBBFE07E92582F8AC
:100AA800020B80E58229F582E5833AF583020B89FA
:100AB800D083D082F8E4937012740193700DA3A3CD
:100AC80093F8740193F5828883E4737402936860E1
:060AD800EFA3A3A380DFE1
:10AAAA00120708601CFF09E970010AC0E0EAC0E069
:10AABA00EBC0E012AC6DD0E0FBD0E0FAD0E0F98058
:0AAACA00DF7F0A12AC6DE4FEFF22EC
:10A3C7008B458A4689478B4B8A4C894DAB45054758
:10A3D700E547AA467002054614F912070870ED749E
:10A3E700FF2547F54774FF3546F546AB48054AE56F
:10A3F7004AAA497002054914F9120708FFAB450537
:10A4070047E547AA467002054614F9EF12074E7052
:08A41700DAAB4BAA4CA94D225F
:10A522008B458A468947E4F54DF54EE54C154CAE10
:10A532004B7002154B4E6033AB48AA49A94A120729
:10A5420008FFAB45AA46A947054EE54EAC4D700241
:10A55200054D14F5828C83EF120760EF60CD740114
:10A56200254AF54AE43549F54980C0AB45AA46A9D2
:02A5720047227E
:10000E00E4FFFE120708600C0FEF70010E09E97095
:05001E00F20A80EF2250
:10ABBE00E94A4B700122120708FF6D700122EF70F7
:0CABCE0004FBFAF92209E970ED0A80EAA4
:100ADE00EF4E6012EF60010EEDBB010B89828A832F
:100AEE00F0A3DFFCDEFA2289F05007F709DFFCA93C
:0C0AFE00F022BBFEFCF309DFFCA9F02293
:109D860002AD07E493A3F8E493A34003F68001F23F
:109D960008DFF48029E493A3F85407240CC8C333DE
:109DA600C4540F4420C8834004F456800146F6DFAD
:109DB600E4800B010204081020408090A81AE47E7B
:109DC600019360BCA3FF543F30E509541FFEE493A2
:109DD600A360010ECF54C025E060A840B8E493A369
:109DE600FAE493A3F8E493A3C8C582C8CAC583CA94
:109DF600F0A3C8C582C8CAC583CADFE9DEE780BE4C
:01A856000001
:100B0A00C5F0F8A3E028F0C5F0F8E5821582700276
:060B1A001583E038F02213
:0C0B2000E2FC08E2FD08E2FE08E2FF2211
:100B2C00E493FC740193FD740293FE740393FF220F
:0D0B3C00E2FB08E2F908E2FA08E2CBF82239
:0C0B4900ECF208EDF208EEF208EFF222E8
:100B5500D083D082E493F208740193F2087402936F
:090B6500F208740393F2740473A6
:090B6E00E6FB08E6FA08E6F922AC
:090B7700E0FBA3E0FAA3E0F9227F
:090B8000E2FB08E2FA08E2F922A6
:0C0B8900E493FB740193FA740293F922C8
:00000001FF
